:10000000981900200D1000006D550000F90F000038
:10001000F90F0000F90F0000F90F0000F90F0000C0
:10002000000000000000000000000000711100004E
:10003000F90F00000000000009110000F90F000096
:100040000913000009130000091300000913000040
:100050000913000009130000091300000913000030
:100060000913000009130000091300000913000020
:100070000913000009130000091300000913000010
:10047C0053B94AB9002908BF00281CBF4FF0FF31FF
:10048C004FF0FF3000F00CB8ADF1080C6DE904CE64
:10049C0000F008F8DDF804E0DDE9022304B0704751
:1004AC00704700BF2DE9F04786468C460846089EEB
:1004BC00154674461946002B40F0C1808542B2FAAD
:1004CC0082F245D94AB1C2F1200300FA02FC9540F0
:1004DC0094402EFA03F343EA0C0C4FEA154EA8B2E3
:1004EC00230CBCFBFEF80EFB18CC08FB00F943EA0E
:1004FC000C43994528D9EB1808F1FF3704D29945DC
:10050C0002D9A8F102072B44A3EB0903A4B2B3FB55
:10051C00FEFC0EFB1C330CFB00F044EA0344A0422F
:10052C0014D92C190CF1FF3304D2A04202D9ACF12E
:10053C0002032C44241A43EA07401EB1D440002382
:10054C0034607360BDE8F0874746DDE76346F1E74A
:10055C0092BB431B01214FEA154EAFB2200CB3FBEB
:10056C00FEFC0EFB1C330CFB07F840EA03439845DA
:10057C0061D9EB180CF1FF3004D2984502D9ACF1DB
:10058C0002002B44A3EB0803A4B2B3FBFEFC0EFB4E
:10059C001C330CFB07F744EA0344A7424DD92C1932
:1005AC000CF1FF3304D2A74202D9ACF102032C4464
:1005BC00E41B43EA0040C0E7C2F12003954094409D
:1005CC0020FA03F12EFA03F34FEA154E9040AFB226
:1005DC000343B1FBFEFC0EFB1C10190C0CFB07F8C3
:1005EC0041EA0041884522D969180CF1FF3004D248
:1005FC00884502D9ACF102002944A1EB08019BB259
:10060C00B1FBFEFC0EFB1C110CFB07F743EA01438C
:10061C009F420ED9EB180CF1FF3104D29F4202D944
:10062C00ACF102012B44DB1B41EA004193E760462D
:10063C00E3E76146F7E76046A4E76346B8E7834221
:10064C0006D916B9002108467CE7C6E900E0F9E7AF
:10065C00B3FA83F78FB9834201D3724508D8BEEB46
:10066C00020460EB030301209C461EB9002169E7DC
:10067C003846FAE7C6E9004CF8E7C7F1200CBB4056
:10068C000EFA07F522FA0CF42EFA0CF1BA401C43C0
:10069C0020FA0CF3B8404FEA144901431FFA84FEC8
:1006AC00B3FBF9F809FB18300B0C08FB0EFA43EA04
:1006BC0000439A4540D9E31808F1FF3004D29A451B
:1006CC0002D9A8F102002344A3EB0A0389B2B3FBBD
:1006DC00F9F809FB183308FB0EFE41EA03418E457D
:1006EC002CD9611808F1FF3304D28E4502D9A8F138
:1006FC000203214443EA0040A1EB0E01A0FB029847
:10070C004145CE46434602D306D14D4504D201386D
:10071C00B9EB020E68EB0403002EA7D0B5EB0E026A
:10072C0061EB030101FA0CFC22FA07F3F9404CEAE5
:10073C000303C6E9003199E74046C5E74346D9E7CC
:10074C00014804F035BD00BF90700000F8B52F488B
:10075C0005F080FB002856D04FF4D0112C4804F043
:10076C0008FD00284FDB2B4805F074FB00284AD00D
:10077C00294D284605F06EFB0446002843D04FF463
:10078C00B011264804F0F5FC00283CDB4FF4803116
:10079C00234804F0EEFC002835DBAE68B769002F67
:1007AC0031D02B694FF0A0721B68012113F0020F9E
:1007BC0014BF4FF000734FF080632846B8470028F1
:1007CC0021DB1849184B4B6002238B60F36913B182
:1007DC000122284698470E4F144E154D384604F00A
:1007EC00E7FC00280FDB84F0010414F0FF0414BFB5
:1007FC00314629460F4804F04FFA002147F61220E3
:10080C0005F0C7FBEAE70020F8BD00BF5067000009
:10081C0098700000346700001867000090700000AA
:10082C0088700000000500204D070000E8710000F2
:10083C00EB710000EF710000014B1B68184700BF03
:10084C00F0000020014B1860704700BFF000002042
:10085C0030B585B004460D4610220021684605F0DF
:10086C00A3FE02238DF80230044B2A46214668462B
:10087C00019304F023FA05B030BD00BF4508000019
:10088C0080B505460E461746984603F0B9F8034660
:10089C0005F0F4FE0446DFF81890424649F80030A3
:1008AC0039463046A84754F8090000F011FC00BF47
:1008BC00080000002DE9F047058B044628079046F8
:1008CC0011D4022905F0070540F0CC80204604F035
:1008DC0067FD78B10138218B042811D8DFE800F0CE
:1008EC00C2106D85950001290CBF45F0100545F02F
:1008FC002005258388F31188BFF36F8FBDE8F0873F
:10090C0001F0070AAA4500F0A5800027B9463E462B
:10091C00A368002B00F0BC8041F00801218388F310
:10092C001188BFF36F8FA168002900F0BA800D68A1
:10093C00002900F0B680334652462046D1F8048098
:10094C00C047002D76D02B6829461D46F0E701F0F4
:10095C0007035A1F012A1BD8002221F00701062B7E
:10096C00276889B2C4E9002209D13B4603E0628BB7
:10097C00013262831B68002BF9D141F00201204641
:10098C00218304F00DFD00287AD041F0200176E09F
:10099C00042B0AD121F0070189B22046218304F0EF
:1009AC00FFFC10B141F020012183218B01F0070ADB
:1009BC00AA454FD00027B946AAE7236921F00701C1
:1009CC0041F00601062DD3F8009021832DD1B9F109
:1009DC00000F3FD041F00801218388F31188BFF349
:1009EC006F8F20463949C84729E021F00701236958
:1009FC0041F0040189B2042DD3F804902183E6D090
:100A0C0000274FF0040A3E4682E721F007012369D4
:100A1C0041F0050189B2052DD3F808902183D6D079
:100A2C0000274FF0050A3E4672E700274FF0060AF2
:100A3C003E466DE72B4687E7B9F1000FD1D1EFF3B6
:100A4C001188202383F31288BFF36F8F238B23F03D
:100A5C0008032383258BEA062ED525F01003238368
:100A6C0005F007056669218B002EBFF670AF0023D9
:100A7C002768C4E9003321F0070141F0010121830B
:100A8C00218B4FF0000901F0070AAA457FF440AF13
:100A9C00002F9CD041F00801218388F31188BFF30B
:100AAC006F8F002FC8D03D683946334652462046DA
:100ABC0004F0A2FC2F46F4E7AB067FF51BAF25F044
:100ACC002003238305F0070500E700BF3154000025
:100ADC00014B036000207047A070000008B504486B
:100AEC0004F051FC034804F04EFC002008BD00BF8C
:100AFC00FE7100003372000008B50348034A002160
:100B0C00121A04F025FD08BDC8020020540C002068
:100B1C00074808B5074A0849121A04F01BFDBDE83E
:100B2C0008400648064A0749121A04F013BD00BFD4
:100B3C0060000020C8020020147700006000002034
:100B4C00600000201477000038B505460C4699B1BA
:100B5C00D1E901230F48096804F015FCD4E90423FA
:100B6C00E1680D4804F00FFCE1690C4804F00BFC43
:100B7C00A1690B4804F007FC012D05D1EFF30581A9
:100B8C000848103904F0FFFB21462846BDE83840E0
:100B9C0002F024BA6172000091720000C172000070
:100BAC00D17200000073000030BFFFF7FDBF00BF23
:100BBC002DE9F04105460B4EDFF82C80324606EB52
:100BCC000807CC1B2046094905F0E1FCA019424658
:100BDC000021083C05F0E8FCC5F8804007F108004E
:100BEC00BDE8F08100000000040000004C70000023
:100BFC00054B5A699B689A421FBF044A536843F0DD
:100C0C0080535360704700BFE405002000ED00E006
:100C1C0010B5204C204804F0B6FBA36A990137D5D7
:100C2C001E4804F0B0FB1E20A36ADA0103D51C4851
:100C3C0004F0A9FB1F20174CA36ADB0203D519484B
:100C4C0004F0A1FB0220A36A1C0303D5164804F090
:100C5C009AFB21200F4CA36A590303D5134804F0C7
:100C6C0092FB2220A36A9A0303D5114804F08BFB54
:100C7C002320084CA36ADB0303D50E4804F083FB46
:100C8C002420A36A6FEA03436FEA1343A36210BDE7
:100C9C001D20C9E700ED00E0147300002D73000067
:100CAC00417300005C73000087730000A6730000A2
:100CBC00CC730000E773000070B5244C0646244842
:100CCC000D4604F060FBA36AD90435D5214804F025
:100CDC005AFB1720A36A1A0503D51F4804F053FBCF
:100CEC0018201A4CA36A9B050FD51C4804F04BFB2B
:100CFC00A16BA36A180407D5194804F044FB1EB174
:100D0C00A36A23F40043A3621920104CA36A59056B
:100D1C0003D5144804F037FB1A20A36ADA050DD565
:100D2C00114804F030FB1B20084A936A43F47F43BC
:100D3C00936200232B7070BD1620CBE7A36A9B0433
:100D4C00F2D50A4804F01FFB1C20EDE700ED00E093
:100D5C00137400002A7400003C74000050740000EE
:100D6C006A740000807400009C740000B57400006C
:100D7C0070B5264C064626480D4604F004FBA36AC3
:100D8C00D80640D5234804F0FEFA1120A36A1907AF
:100D9C0003D5214804F0F7FA12201C4CA36A9A07D9
:100DAC000FD51E4804F0EFFA616BA36A1B0607D53A
:100DBC001B4804F0E8FA1EB1A36A23F08003A36277
:100DCC001320124CA36ADE0703D5164804F0DBFA95
:100DDC001420A36A9C0603D5134804F0D4FA1520FA
:100DEC000A4B9A6AD10658BF9A6A9A6A920642BF0F
:100DFC005A6A22F400525A629A6A42F0FF029A62CC
:100E0C0000232B7070BD1020C0E700BF00ED00E088
:100E1C00E5740000FC7400003C74000030750000A8
:100E2C004975000060750000B57400002DE9F041B3
:100E3C005B4B04465F6800258AB0C7F3080685F350
:100E4C001188BFF36F8F02F07F43B3F17F4F06D150
:100E5C0002F00C03082B13D1524804F094FA00252D
:100E6C002C464FF00008F31E8DF80780092B00F27A
:100E7C008580DFE803F00A797D7583838383838122
:100E8C0010074CBF0C460125EBE74748444E04F0D5
:100E9C007AFA8DF80780F36A9A0704D5434804F070
:100EAC0072FA00232FE0F36A002B01DA4048F6E7D0
:100EBC00F36A5B00F5D53F4804F065FA7369A269E3
:100ECC0043F480737361BFF34F8FBFF36F8F7369FC
:100EDC0032F8022C23F480737361BFF34F8FBFF38E
:100EEC006F8F4DF602739A4208D0B36ADBB24BB3E4
:100EFC0001200DF10701FFF73BFF33E021682E487D
:100F0C0004F041FA23689DF80720C2B902AE04F13F
:100F1C002007324620686168083403C2BC4216467A
:100F2C00F7D1099AB5B3C2F3080121B96FEA52227D
:100F3C006FEA42220992184602A9FFF705FE0AB091
:100F4C00BDE8F081B36A13F47F4F05D001200DF199
:100F5C000701FFF7B1FE05E0B36AB3F5803FA0D3FC
:100F6C00FFF756FE0346CEE700200DF10701C2E75E
:100F7C0000200DF10701ECE7104890E7104B17F437
:100F8C00F87F1049104818BF1946A6F1100204F05A
:100F9C00FAF986E722F4FF7222F00102CAE700BFD9
:100FAC0000ED00E0AE750000DA750000F27500008F
:100FBC001476000023760000437600006076000073
:100FCC00957500008075000085760000064B5A6907
:100FDC0042F010025A615A6942F480625A615A69AD
:100FEC0022F008025A61704700ED00E0EFF3088030
:100FFC00EFF3098101B57246FFF718FF01BD00BF81
:10100C00002080F31488BFF36F8F002080F30A88D0
:10101C0080F30B880F4880F3088801F089F90020D1
:10102C000D490860BFF34F8F00F02CF8202080F39F
:10103C0011880A484FF40061401880F30988EFF3D7
:10104C0014800221084380F31488BFF36F8F00F0E3
:10105C00EFF800009819002094ED00E0580C0020E7
:10106C00002318460649D1F89020C2F30722934278
:10107C0000DB7047C1F89830C1F8A0000133F6E7E7
:10108C0000ED00E010B572B6002484F31388FFF76E
:10109C00E7FF23464FF0FF300C4A03F120010133E8
:1010AC00102B42F82100F8D100234FF0FF30074AF3
:1010BC0003F160010133102B42F82100F8D162B624
:1010CC00BFF34F8FBFF36F8F10BD00BF00E100E087
:1010DC00084B9B6883420BD1EFF3058343B1064B5E
:1010EC005A6842F080525A605A6A22F400425A629C
:1010FC0002F08CBCE405002000ED00E016498A6883
:10110C004FF030001044EFF3098C80E8F01F2020E2
:10111C0080F31288BFF36F8F104F4FF000664A694F
:10112C008A603E60D2F880000D4C2060D2F88400BA
:10113C000023C2F8843080F3118802F1300090E86B
:10114C00F01F8CF3098802F1000004B504F013FAC7
:10115C00BDE8044070470000E405002004ED00E009
:10116C000C0500201EF0040F0CBFEFF30880EFF30A
:10117C000980816911F8021C0229FFD001B5724661
:10118C0004F0EAF901BD00BF00B2002807DB01231F
:10119C004109034A00F01F00834042F82130704798
:1011AC0000E100E000B200280CDB012206494309F3
:1011BC0000F01F008240203341F82320BFF34F8FF3
:1011CC00BFF36F8F704700BF00E100E0054B420991
:1011DC0053F82220012300F01F0003FA00F0104006
:1011EC00704700BF00E100E000B2002801F10101EE
:1011FC00ACBF00F16040064B4FEA4111C9B2ABBF26
:10120C0000F5614000F00F0080F80013195470478E
:10121C0014ED00E0044B054A23F07F039360BFF309
:10122C004F8FBFF36F8F70470000000000ED00E0A0
:10123C0008B5FFF7EFFF074AD2F8883023F47003A4
:10124C00C2F88830FFF758FCFFF762FC00F046F854
:10125C0001F088FF00ED00E042F8203C009B0B49B8
:10126C0042F81C3C019B21F0010142F8183C029B06
:10127C0042F8081C42F8143C4FF0807342F8043CCE
:10128C000023203A0265C0F8843070478D080000B6
:10129C0000B50D4B15469860D0F880200B4B0E46D0
:1012AC001A60036F83F30B882C4686F309880020A1
:1012BC00034B98472046002100220023014C204775
:1012CC00915500008D080000E40500200C0500205D
:1012DC001022014B1A61704700ED00E00023202022
:1012EC0040F20F1210B5044CE1180133934281F80F
:1012FC000003F9D110BD00BF00E100E008B5EFF329
:10130C000583064A103B02EBC30152F833004968CF
:10131C008847BDE80840FFF76BBC00BF886700003A
:10132C001FB5094C094A23460121094800F0FAF877
:10133C0000230393074B0121E41A01A801930294A3
:10134C0000F0FAF804B010BD00F0022000000020FC
:10135C00A0700000C802002010B50C7A0B6804F0D5
:10136C001F0223F01F031A43CB68640923F01F03E9
:10137C00054943EA440343F00103C1F89800C1F85E
:10138C009C20C1F8A03010BD00ED00E010B5074B5B
:10139C00D3F89030C3F30723013B984202D8FFF7F0
:1013AC00DBFF10BD6FF01500FBE700BF00ED00E0A8
:1013BC002DE9F04F0F46144606464FF000084D4DF0
:1013CC0085B0B84580F29280D6F80490B9F1000F40
:1013DC0036D0B9F11F0F40F2878019F01F0F40F083
:1013EC008380D6F800A01AF01F0F7DD1504604F070
:1013FC00ECF8834609EB0A00013804F0E6F8834563
:10140C0072D11BF1160F6FD05C456DDDC5F898B02D
:10141C00D5F89C10C5F898B0D5F8A03021F01F0174
:10142C0043F01F0AD6E900321A44994202F1FF39FF
:10143C001ED1CA4508D131465FFA8BF004F0CEF8C4
:10144C0008F101080C36BCE73146C5F898B0D5F860
:10145C009C3022F01F0203F01F031343C5F89C308D
:10146C00E0B204F0BBF810F1160F3DD0441CE7E7D6
:10147C00C5F898B0D5F8A020013B23F01F0302F06B
:10148C001F021343CA453146E0B2C5F8A030E8D07C
:10149C0004F0A4F810F1160F26D0C5F898B0D5F8C2
:1014AC009C209DF808300AF1FF3A62F304038DF892
:1014BC000830D5F8A0309DF808205B0863F347127C
:1014CC008DF80820D6E900321344009323F01F0353
:1014DC005344A3EB0903013023F01F036946C0B248
:1014EC000393FFF753FFBEE76FF01504204605B0DA
:1014FC00BDE8F08F00ED00E00522044BC3F894200A
:10150C00BFF34F8FBFF36F8F704700BF00ED00E04C
:10151C00BFF35F8F0022024BC3F89420704700BFCB
:10152C0000ED00E010B5034C2278FFF741FF20706E
:10153C0010BD00BF4C0C00202DE9F74F294D8A46F9
:10154C0006464FF00008AB46274FD0451BDAD6F8BD
:10155C000490B9F1000F3FD031680846019104F0B6
:10156C0034F80199044609EB0100013804F02DF818
:10157C0084424FF014021D4B08D002FB08F36FF0AD
:10158C0015024BF8032003B0BDE8F08F14F1160FD1
:10159C002C60F8D01978A142F5DD02FB08B0C7F831
:1015AC009840C7F89840D7F89C4000F10801007BA0
:1015BC0064F304000871D7F8A0000C79400860F3BC
:1015CC0047140C71D7F89C1021F01F016960D7F8F3
:1015DC00A01021F01F01296108F1010814350C3607
:1015EC00B3E700BF1005002000ED00E04C0C00201C
:1015FC00F0B55249524CD1F890302568C3F307230B
:10160C009D4287B000F296800020FFF781FF4D4B82
:10161C00C1F8C030854216D14B4C01A82570FFF79C
:10162C0057FA00250646494FAE4213D100202378C5
:10163C004249D1F89020C2F30722934274DBFFF7A2
:10164C005BFF002043E0616801EB0011FFF784FEB3
:10165C000130DFE70199280101EB0513DA683A4004
:10166C00B2F5800F42D007D8B2F5801F15D0B2F575
:10167C00001F2ED00135D7E7B2F1006F43D0B2F185
:10168C00805FF7D15A689B680958013B22F01F0014
:10169C00034423F01F03012032E05A689B68095869
:1016AC00013B22F01F0003440120844623F01F035A
:1016BC0040EA4C10CDE902218DF8100002A92078E7
:1016CC000593FFF763FE00282ADA6FF0150007B0C8
:1016DC00F0BD5A689B680958013B22F01F00034477
:1016EC004FF0020C012023F01F03E1E75A689B68BE
:1016FC000958013B22F01F000344062023F01F036E
:10170C004FF0000CD4E75A689B680958013B22F053
:10171C001F0003444FF0030C012023F01F03C7E705
:10172C00237801332370A5E7C1F89830C1F8A000E5
:10173C0001337EE74FF0FF30C9E700BF00ED00E05A
:10174C00AC700000AAFF44004C0C00200000F0FF1D
:10175C0008B5024B1B689847002008BD24050020E3
:10176C00034B044A1860937843F00203937070475C
:10177C0024050020F400002008B50649064821F095
:10178C000701C1F1005202F53C3203F0A2FD00202A
:10179C0008BD00BF9F1900202805002008B5244A69
:1017AC00244B1A6000F060F84FF47A612248D0F8AC
:1017BC002436C3F30802C3F309434B4382F480720B
:1017CC001E49883201FB02334FF4FA215B00B3FB54
:1017DC00F1F201FB12331A49B3F57A3F28BF0132FB
:1017EC00C1F80429D0F820364FF47A60C3F308020C
:1017FC00C3F30943434342F21C5082F4807202F259
:10180C00172200FB02334FF47A701B0AB3FBF0F281
:10181C0000FB12330020B3F5FA7F4FF0010328BF11
:10182C000132C1F81C27C1F80009C1F8003608BD07
:10183C000020A1070002002000C0FF00F82A008051
:10184C000000125048B1054B054A1B68B3FBF2F37C
:10185C005843044B43F00103184770470002002023
:10186C0040420F00707000000122024BC3F80424A8
:10187C00704700BF002008E0084B70B5C31A0D4636
:10188C0007499B10044659434022064803F0CDFEFD
:10189C002B4601462046BDE87040184748050020FD
:1018AC00B76DDBB6FC660000402373B50B4C0093A0
:1018BC00041B0B460D460A49A41061430646094A0F
:1018CC00094803F0DEFE011E05DA30462B4602B055
:1018DC00BDE87040184702B070BD00BF480500203D
:1018EC00B76DDBB6F9560000FC660000F8B50022B7
:1018FC000121054640F20510FFF776FC0F4800F079
:10190C00B7FD0446B8B900F0D3FD2F690C49384631
:10191C0003F095FD031E09DB01263E642D69084981
:10192C0005F11C0003F08BFD031E02DA1C46204659
:10193C00F8BDEE64FBE76FF00404F8E77D1A0000D5
:10194C00D87000001FB500220123CDE902236B469D
:10195C00084ACDF800D0CDF804D003F0C0FE002822
:10196C0005DB43F609520023684601F05DFD05B026
:10197C005DF804FB0B57000010B5EFF31184202326
:10198C0083F31288BFF36F8F074A136823F00201A9
:10199C00DB07116002D4012003F0F4FF84F31188FB
:1019AC00BFF36F8F10BD00BF980500200C22104BA9
:1019BC00014602FB0033002030B4D3E90E52986389
:1019CC00EFF31180202484F31288BFF36F8F1C6C0B
:1019DC0004F0C00444F002041C6480F31188BFF3CB
:1019EC006F8F1DB12B4630BC0248184730BC704776
:1019FC0048050020FC66000010B4EFF31182202390
:101A0C0083F31288BFF36F8F1648016841F002040C
:101A1C000460C80707D482F31188BFF36F8F0120CD
:101A2C0010BC03F0A7BF1049D1F80C14C903F2D5B0
:101A3C00EFF3118083F31288BFF36F8F0B490B6C9C
:101A4C0003F0C00343F002030B6480F31188BFF36F
:101A5C006F8F82F31188BFF36F8F002010BCFFF7DC
:101A6C00A5BF00BF9805002000E0105048050020DD
:101A7C00022808D0042808D1044B186C10F0070079
:101A8C0003D1FFF793BF0120FBE770474805002007
:101A9C002DE9F041012207463449D1E8EF3FC1E876
:101AAC00E02F0028F9D133B9314932484B60CB6073
:101ABC008A6003F0D7FC7B1E012B28D8012F06D19E
:101ACC002D4BD3F8503403F00303012B1FD004F03B
:101ADC00EAF90546E8B9294B1B78D3B1042206462E
:101AEC00254BC3F80823244CDFF89480D4F84C24FD
:101AFC00D4F84C34D20315D503F00303012B01D0D9
:101B0C00012F0FD165B386F31188BFF36F8FBDE83A
:101B1C00F081EFF31186202383F31288BFF36F8FCC
:101B2C000125E0E7BDB1304603F040FDD4F8403468
:101B3C0013F0FF03DAD1D4F80821002AD6D0C4F868
:101B4C000831D4F8083120220123C4F84034C8F8F5
:101B5C00A0212361CAE70021202004F01AFAE5E74E
:101B6C000422054BC3F80423D1E700BF4405002031
:101B7C00340500206405002000E010504F0C0020BC
:101B8C0000E100E008B5074804F064F938B10648F4
:101B9C00FFF7E6FD0448FEF755FE002008BD6FF088
:101BAC001200FBE76C670000B91B00000A2838B56F
:101BBC000446074D04D1AB680D2128465B68984755
:101BCC00AB6803485B68E1B29847204638BD00BF5C
:101BDC006C6700002DE9F04340F206354768D006EB
:101BEC0048BF4FF0030C3B7C02EA050558BFC2F31B
:101BFC00401C87B001F01F06B5F5837F144646EAFA
:101C0C0043168DF803C046D00DD8062D45D005D807
:101C1C00A5B1022D12D06FF0150039E0B5F5807F1B
:101C2C00F9D101250AE040F20222954237D0B5F5F0
:101C3C00407F36D0B5F5007FEDD10425012322037A
:101C4C0003FA01F12FD57B685960B86880BB5F2E11
:101C5C0006F01F034FEA561173D83C4A52F8212064
:101C6C0084F4803102EB8302D2F88030C1F300415E
:101C7C00C4F3404423F4706344EA410423F00F039B
:101C8C001C4344EA8C0444EA0524C2F8804000203A
:101C9C0007B0BDE8F0830925D0E70825CEE7062577
:101CAC00CCE70525CAE7630344BF7B689960CCE7A2
:101CBC0031460DF1020204F03FF814F4403F804627
:101CCC000CD13146B86804F050F8B8F1000FDED1F1
:101CDC009DF80210B86800F07DFED8E74FF00009BF
:101CEC0001ABCDE90199CDE90439CDF80C90314621
:101CFC00B86803AA03F064FF4845C8DB14F400334A
:101D0C0014D09DF8033084F48034C4F300448DF86F
:101D1C000E308DF80C508DF80D404B463146B8689E
:101D2C0003AA00F0A5FD0028CFDAB0E7CDE9043313
:101D3C000DF1030303933146B86803AA03F040FF87
:101D4C00F1E7203350F82330FFDE00BFF4700000C1
:101D5C004209022A034670B503D0012A18D0CAB131
:101D6C0070BD0E4E326951680029F9D0012503F07F
:101D7C001F030C689D400029F2D08A682A4002D0CB
:101D8C0030464B6898473CB1236821461C46F2E725
:101D9C00034EE7E7034EE5E72346F6E750670000FE
:101DAC00346700001867000038B54568A868C0B1F2
:101DBC0003F0D5FF0146A0B9A86800F0D3FD044696
:101DCC0088B902460949A86803F0B3FF22460121ED
:101DDC00DB20FFF709FA2246012140F20D10FFF734
:101DEC0003FA002038BD6FF00400FBE75D1D000016
:101DFC00F0B544681646A068227C01F01F0587B038
:101E0C0045EA421500286CD0B6F5001F04D12946CE
:101E1C0003F0FFFF002055E06268607CB6F5800F90
:101E2C0050624FF0000001AA0190506039D1B3F11B
:101E3C00007F14BF052304238DF804300023CDE963
:101E4C0004230393E3680DF1030723FA01F111F066
:101E5C00010139D1B6F1A07F36D105F01F035F2DFA
:101E6C004FEA551003F120033ED8214A52F82020A6
:101E7C0052F82330DB0727D43A462946A06803F0F2
:101E8C005BFF163018D002972946A06803AA03F00E
:101E9C0097FE002816DB01222946A06803F067FF95
:101EAC00B8E7B3F1C06F05D0B3F1007F14BF0123C5
:101EBC000223C1E70323BFE73946A06800F094FD75
:101ECC000028E0DA07B0F0BD3A462946A06803F0D6
:101EDC0033FF0028D8D19DF80310A06800F07AFDDC
:101EEC00D2E76FF08500EDE751F82330FFDE00BF3D
:101EFC00F4700000036803F01F025F2B02604FEACE
:101F0C0053129ABF024B53F822000020704700BFB7
:101F1C003C7100002DE9F04F1546074640F2FF19C1
:101F2C00DFF868A1DFF868B185B000EB8101B94238
:101F3C0003D1002005B0BDE8F08F3A68C2F3C3238B
:101F4C00082BC2F3080400F29E804C4508BF4FF0EA
:101F5C00FF34B2F1D05F1AF803804FEA126310D24B
:101F6C00192B12D8DFE803F014226461292F6111B8
:101F7C00111111111111111111111111111167718F
:101F8C007477382B6AD04E2B52D06FF08500D1E786
:101F9C00C5F80446601C14D0012603A80394FFF76F
:101FAC00A9FF039B06FA03F3436004E0C5F80C4653
:101FBC00621C06D00026324613E0631CC5F80046AE
:101FCC005FD10437B3E7661CC5F80446F9D0012687
:101FDC0003A80394FFF78EFF0122039B02FA03F37D
:101FEC0083603B68039403F40040002818BF002270
:101FFC0003A818BF012601930092FFF77BFF039CF7
:10200C00019B00EB8400D0F88040C3F3412C009A74
:10201C004FEA082343EA8C03134304EA0B042343DB
:10202C0043EA4603C0F88030CBE7C5F80846BFE763
:10203C00C5F81046AEE7C5F86045621C3B68C0D0D9
:10204C00C3F30043002BC2D0A6E7C5F86445F4E700
:10205C00C5F86845F1E7C5F86C45EEE703A80394AD
:10206C00FFF748FF039B00EB8300D0F8803023F090
:10207C00E04343F08043C0F88030631CA1D00126BC
:10208C0099E70026A4E76FF0150053E7D776000018
:10209C00F0F0FCFF2DE9F04104460D46476803F0D3
:1020AC0002FF88B12021EFF311831A4681F31288C5
:1020BC00BFF36F8F60680068D0F83001D0B983F33C
:1020CC001188BFF36F8FEEE71E4B1B78002BE9D006
:1020DC004FF02008642663681B68D3F83031FBB9D5
:1020EC00012003F010FC013EF5D10021202003F06B
:1020FC0050FFEFE77B6A00201D706368796A1B68EC
:10210C00C3F83C170121C3F84017C3F83001D3F8CA
:10211C003001196582F31188BFF36F8FBDE8F08130
:10212C00EFF311831A4688F31288BFF36F8F61683F
:10213C000968D1F830110029DCD183F31188BFF381
:10214C006F8FD2E74F0C002070B40D4CD4E90065B2
:10215C00901B63EB0501400940EAC16041018919FC
:10216C0045EBD065C4E90015002400250549C1E9FB
:10217C000023054BC3E9004570BC01F027BE00BF2E
:10218C00E8020020D0020020E002002008B5002266
:10219C000121E420FFF728F8164A0020D2F818375E
:1021AC0023F44033C2F8183700F07EFD002820DB02
:1021BC000120114900F004FE00281ADB00F04EFD4E
:1021CC000E4B20F01F00C3E900010D4B0022C3E9A8
:1021DC0000014FF0FF304FF0FF310A4BC3E9000113
:1021EC00094B0A49187A00F049FD67220020084B78
:1021FC001A6008BD00200E50FC010020E8020020EF
:10220C00C8020020D0020020F4010020552100005B
:10221C00C805002008B500F021FD064AD2E90032BD
:10222C00C01A054B61EB0201C3E90001400940EA09
:10223C00C16008BDE8020020E0020020F7B5224B87
:10224C000146224F187A224BD7E90056D3E90023D6
:10225C009E4208BF954211D1B1F1806F0ED2490157
:10226C00012938BF012101224D1946F10006C7E9A9
:10227C00005603B0BDE8F04000F02CBE154BDFF863
:10228C0058C0D3E90043DCE9002CA41843EB0C0C38
:10229C004FF0200E22466346C1FB0E23954276EB8F
:1022AC000301C7E900230DD2291B66EB0C04C829D6
:1022BC0074F10004B4BF01210021009100F0D2FDA3
:1022CC0003B0F0BD0021F8E7F4010020D802002093
:1022DC00D0020020E8020020E0020020064BD3F8D8
:1022EC0040231C2A05D1D3F84403431E58425841BD
:1022FC0070470020704700BF00C0FF0003689A07BA
:10230C000CD50368DB070DD50922074BC3F80C2548
:10231C000F22C3F8042501221A60FEE7034B036069
:10232C00EF3B0360704700BF00801050F000FA5084
:10233C0008B50123404A4148C2F80038404AD2F857
:10234C0040231C2A04BF3F4AC2F80C34FFF7D6FFC7
:10235C000830FFF7D3FF0830FFF7D0FF0830FFF746
:10236C00CDFF00F5F470FFF7C9FF374AD2F88C3077
:10237C0043F44063C2F88C300022D30003F57F0392
:10238C0003F54043D3F8001401310AD0D3F80014FC
:10239C0039B1D3F800140132D3F80434402A0B605D
:1023AC00EBD1254BD3F84024002A41D0FFF796FF00
:1023BC0048B1234BD3F83423244B9A429EBF1E4B77
:1023CC00234AC3F84026FFF789FF18B1214B224A54
:1023DC00C3F8AC27FFF782FF48B13422164BC3F881
:1023EC002426D3F83C2622F40022C3F83C261B4BAF
:1023FC001549D3F80026D20744BF6FF00102C3F889
:10240C000026174BD3F8182522F00302C3F8182521
:10241C00D3F8182542F00302C3F81825D1F88C2004
:10242C0042F44062C1F88C200022C3F8A02508BDFC
:10243C00C822C3F84024B9E70000125000C50D5063
:10244C0000C0FF000030055000ED00E0001D0A1830
:10245C0040E0A91E00A0085078000A0400E01050CB
:10246C0000B00450014B1B68184700BFCC0500207E
:10247C0010B50C4C237993B9012323710A4B002816
:10248C00206018BF184600F0F3F850B923680748CD
:10249C00002B08BF1846BDE8104000F035B86FF0AF
:1024AC00770010BDCC050020712400007D59000080
:1024BC0008B5074B1B6853B140F20510FEF786FEBA
:1024CC0028B9BDE8084040F20510FEF75DBE08BD16
:1024DC00CC05002038B504230A4C42F21075C4F820
:1024EC000833012363610023C4F80831D4F80831A0
:1024FC00D4F84C34DB0304D5012003F004FA013D7D
:10250C00F6D138BD00E01050064A13793BB90121D1
:10251C0010601171044A1846C2F8403470476FF0CD
:10252C0077007047D405002000E0105010B51D4B0B
:10253C001D4CD3F84C14D3F84C2411F4803F18D014
:10254C0002F00302012A03D00AB1FFF7C3FF0022F5
:10255C00144BC3F840240022C3F80821D3F80821F7
:10256C0001221A61226872B9D3F80821002AFBD023
:10257C0011E0D3F84824D107E9D5D3F850249207B9
:10258C00E3D422681AB10422C3F8042310BDD3F893
:10259C000821002AFBD00022C3F80821D3F8083107
:1025AC00F4E700BF00E01050D4050020F8B5012579
:1025BC00184C194ED4F80C3303F00C0303B9F8BDC6
:1025CC00B3FA83F30027C3F11F039A0002F580725C
:1025DC0092B202F1A04202F58712176005FA03F1DC
:1025EC00022B1268D8B2C4F8081310D1D4F84C34AA
:1025FC00D4F84C349B070AD10423C4F84054C4F8D3
:10260C0004332561D4F80C3303F00C03D6E733689C
:10261C009847F7E700E01050D4050020712238B538
:10262C00104B0021C3F80823012242F210745A60A7
:10263C00C3F80011D3F800110B490A4DD1F840131F
:10264C001C2908BFDA60D5F80C3413F4803305D09C
:10265C00012003F058F9013CF5D138BD034A537100
:10266C00FBE700BF00E0105000C0FF00DC050020BD
:10267C00054B0246187918B91A6001221A71704775
:10268C006FF07700704700BFDC0500200022164B6E
:10269C00C3F81021D3F81011C3F81821D3F818116E
:1026AC00C3F81421D3F814111049D1F840131C2984
:1026BC0004BF01219960C3F80021D3F80021012245
:1026CC001A600B4A126852B9074BD3F80021002A42
:1026DC00FBD00022C3F80021D3F8003170477122DF
:1026EC00C3F80423704700BF00E0105000C0FF0087
:1026FC00DC050020F8B50126194C1A4DD4F80C3322
:10270C0003F0710303B9F8BDB3FA83F30021C3F1ED
:10271C001F039A0002F5807292B202F1A04202F5F8
:10272C008712116006FA03F7042B1268D8B2C4F8AA
:10273C00087308D0062B10D02B689847D4F80C33AC
:10274C0003F07103DEE702236B71C4F81411D4F8A3
:10275C0014312023C4F80433EEE76971ECE700BFB1
:10276C0000E01050DC050020036803F01F025F2B13
:10277C0002604FEA53129ABF024B53F8220000201A
:10278C00704700BF98710000034A4309D35C00F006
:10279C001F001844C0B27047EB760000F0B5064637
:1027AC00002487B0114F019117F8012B06AB03EBF6
:1027BC00D20313F8143C02F00702D34013F00103C8
:1027CC0006D10134032CEFD10023184607B0F0BD1D
:1027DC00074A03AD07CA85E8070055F824100A6AB2
:1027EC0046F824200A62002AEBD0EEE7FB760000C4
:1027FC0050700000F7B504460846FFF7C5FF06B257
:10280C0004EB4606B38A0D46DB072BD5204603F0B6
:10281C00B4F92946204603F020F958B1204603F0BC
:10282C0032F90022276800B207EB8003C3F81025A9
:10283C00C3F810252946204603F04EF9002101A8C3
:10284C00B1820195FFF790FF019B00EB8300D0F85C
:10285C008020064B134043F00203C0F8803008463A
:10286C0003B0F0BD6FF01500FAE700BFF0F0FCFF0D
:10287C002DE9F043044685B0084616461D46FFF781
:10288C0083FF0F46804636B3204603F0F1F818B9A3
:10289C00204603F0E2F828BB0FFA88F904EB49094B
:1028AC00B9F8143013F01C0F02D07378012B19D027
:1028BC0001238DF80F3000233846CDE90063721CDC
:1028CC00B31C0DF10F0103F070F8B9F8143043F09C
:1028DC000303A9F81430002D40D03946204603F0EC
:1028EC00C7F820B96FF0150005B0BDE8F0830022E1
:1028FC00297823684FEA810C03EB8103C3F8102578
:10290C00C3F810250FFA88F204EB4202938A23F4E1
:10291C00604323F0200393826E78FEB12468A8787C
:10292C006444D4F810550E4B36042B40C4F81035C3
:10293C0041F6F07306F4403603EA07130005D4F8A9
:10294C001055334300F4801003432B43C4F8103567
:10295C00938A43EA413343F0200393820020C3E778
:10296C000FE0ECFF70B590F87440054690F8756078
:10297C0044BB46222146143003F016FE2146134A6E
:10298C002B6852F836608E4212D1002440F20D10A2
:10299C00C3F84441D3F844210D4A934208BFDB20CD
:1029AC00FEF7F2FB0123204685F874302B6670BDD0
:1029BC00CAB2920002F58070442A04BF1C501A5807
:1029CC000131E0E76FF07700F1E700BFA471000080
:1029DC0000A00D5090F87500024B03EB800002F044
:1029EC00AEBF00BF0402002010B5064B90F8750076
:1029FC000C4603EB800002F088FF0028A4BF207077
:102A0C00002010BD040200202DE9F04F814659F83A
:102A1C00043B8BB0D3F8141390F8754000936C4BB7
:102A2C00C9B241F40031804653F83420009803F0C9
:102A3C007DF8810305463AD50023CDE90733099388
:102A4C00634B07A803EBC4035B6819460193FFF7BC
:102A5C00A5FE042303EBC40303934FF0000B5D4B63
:102A6C000DF11C0A0293029A594912F8013B029289
:102A7C00039A02EBD3028A5C03F0070322FA03F3F6
:102A8C00DA071AD40BF1010BBBF1030F0AF1040A9C
:102A9C00E9D14FF400310022009803F047F8019976
:102AAC0007A8FFF77BFE0028D7D125F400350124B9
:102ABC00002D75D10BB0BDE8F08F474B5B440493F0
:102ACC00DAF800100029DDD091FAA1F1B1FA81F108
:102ADC00049B1C7841EA44142046FFF755FE08EB92
:102AEC004000878AC808BB08059301231AF8002008
:102AFC0001F0070103FA01F122EA01020AF80020B1
:102B0C0006A80694FFF730FE069A059B203250F873
:102B1C002220C7F382065B073746C2F3014223D556
:102B2C004846D6B221463A4602F0B7FF06A80694AC
:102B3C00FFF71AFE069B203350F82330C3F30143F2
:102B4C009E4207D10021204602F078FF31462046F4
:102B5C0002F074FF06A80694FFF706FE0122069BFE
:102B6C0002FA03F30362ABE7022A0DD103212046DC
:102B7C0002F064FF06F00503012BEBD13A46214627
:102B8C00484602F08AFFE5E702212046059202F052
:102B9C0055FF032EF2D0059A032ADBD1022EECE767
:102BAC0095FAA5F3B3FA83F3009904FA03F225EA34
:102BBC00020503F5A27251F8222008EB43034846A4
:102BCC00B3F86410C2F3014202F067FF70E700BF74
:102BDC00A4710000FB760000FB7600000123034A81
:102BEC0003FA00F093680343936070476000002081
:102BFC0073B504460191EFF31186202383F31288F9
:102C0C00BFF36F8F0B4D019B6A6801A813400193B2
:102C1C0002F07BFE002807DB01226B68824023EA6E
:102C2C0002036B602070002086F31188BFF36F8F56
:102C3C0002B070BD60000020074B027AD3F810156B
:102C4C0021F001010A43C3F810250268C3F8A42639
:102C5C004268C3F8AC26704700200E504FF0FF328C
:102C6C006FF0404330B5044CD4E90001824273EB61
:102C7C000105F9D330BD00BF40270E5030B50C25EF
:102C8C00074B1C1894F8544005FB0433C3E903129A
:102C9C0018750123034A8340C2F8243330BD00BFAA
:102CAC006000002000200E50F0B53D4D85B02C7812
:102CBC00002C6FD13B4A01AB07CA83E807003A49A5
:102CCC001846D1F8102522F00202C1F81025FFF7A2
:102CDC00B3FF0723672202F001012144013BCCB270
:102CEC004FEA5202F7D1052C57D119464FF0010C7F
:102CFC002B4E00246720CFB204E00CFA02F220EA3B
:102D0C000200013490FAA0F25FFA84FEBE45B2FADA
:102D1C0082F2F2D30131327505292A4482F85470BB
:102D2C0006F10C06E5D10121002420489A0801FA8D
:102D3C0002F212F0670F18BF1C500433302BF5D180
:102D4C00E420FEF721FA184B1949D3F8102503F5A6
:102D5C00C07322F00202C3F8902340F6FF72C3F84E
:102D6C00A82100221A60A3F5807004338B42026004
:102D7C00F8D101240C4B0F4A1C660F4B5D201B68CD
:102D8C00B3FBF2F358430D4B2343984700202C70B0
:102D9C0005B0F0BD6FF07700FAE76FF08B00F7E746
:102DAC00600000205C70000000200E5000210E50CE
:102DBC00B0210E5040420F00000200208070000035
:102DCC0038B5254B0C46D3F8102595073DD4D3F8D0
:102DDC00102542F00202C3F81025C0B1D3F84827E1
:102DEC0012F0010202BFD3F8481741F00101C3F8F9
:102DFC004817194BD3F84017D3F844174900F9D4A6
:102E0C002AB9D3F8482722F00102C3F84827134BFC
:102E1C00134A1B681049B3FBF2F303EB4313BBB12A
:102E2C00D1F84027D1F8445715F080450BD14FF01D
:102E3C00FF312046FFF7DCFE002803DB2078FFF78C
:102E4C00CDFE284638BD013BE9E76FF07700F9E786
:102E5C006FF07300F6E700BF00200E500002002058
:102E6C0040420F0070B51D461446184A9DF810607C
:102E7C00131893F8543000B20C3302EBC30142F830
:102E8C0033404D60C5F31301AEB10201104E02F197
:102E9C00A04202F562228000C2F820450644C2F826
:102EAC002415336833B1FFF7D9FEA042A94101D2F2
:102EBC000023336070BD030103F1A04303F56223CB
:102ECC00C3F82045C3F82415F4E700BF60000020C8
:102EDC0000210E50F0B50E4D2B1893F85430000114
:102EEC000C3355F8334005EBC3077E68641800F1CA
:102EFC00A04021F0004146F1000641EAC27100F504
:102F0C00622045F833407E60C0F82815F0BD00BF44
:102F1C0060000020F7B5284B284CD3F82C6304F143
:102F2C0088070EB903B0F0BD96FAA6F00123B0FAEB
:102F3C0080F08340DA43224926EA0306231893F8EB
:102F4C005450830019440C2303FB0543DB6873B313
:102F5C00D7E8EF3F03EA020CC7E8EECFBEF1000F53
:102F6C00F6D1C340DB0719D5020102F1A04202F5EC
:102F7C006222D2F82435D2F82025D1F800C0BCF159
:102F8C00000FCED04FF0000CC1F800C00C2101FB9B
:102F9C00054529690091E9688847C2E705F10C03EA
:102FAC0004EBC30C54F83320DCF80430E5E70A6872
:102FBC00002AB6D00B60B4E700200E506000002051
:102FCC0000210E50044B40EA0120C3F80005D3F851
:102FDC000024D207FBD5704700B0045038B5EFF38E
:102FEC001185202383F31288BFF36F8F064B9C68E7
:102FFC0002F043FF85F31188BFF36F8F2046BDE8C5
:10300C003840FEF765B800BFE405002038B50A4B20
:10301C0053F82040013053F82050A54200D838BD59
:10302C00606830B1037EDB0701D402F0FBFE08348C
:10303C00F3E723689847FAE7B4710000012270B5F2
:10304C00294B032086B01A70FFF7E0FF03F034F829
:10305C000420FFF7DBFF254C254D2646AE4204F13C
:10306C00300410D300F0D8FB204C224EAC4226D3B7
:10307C0000F0E6FBFDF76AFB1F4A137B23F001030C
:10308C00137306B070BD54F80C3C059354F8103C07
:10309C00049354F8143C039354F8183C029354F8DA
:1030AC001C3C019354F8203C009354E90A2354E946
:1030BC000C0100F0DFF954F8303C5E65CDE7D4E943
:1030CC000A23B3F1FF3F08BFB2F1FF3F05D052EA2C
:1030DC000301206803D100F06FFC3034C6E73146A1
:1030EC00183000F0E3FDF8E74F0C002000700000F2
:1030FC0000700000975F000080030020902370B5E3
:10310C00134E012203FB0066002386B0CDE9042395
:10311C000F220193CDE9023214234FF4A0720D4D0E
:10312C000D4903FB0055044602FB00110B4B3046C6
:10313C00009500F09FF9737B2C7423F004037373D8
:10314C00074B013403EBC423EE606B6006B070BD1B
:10315C00F0020020E4050020581400208D5E0000D1
:10316C00580C0020BFB50020FFF750FF284B03F58B
:10317C00006282F3088883F30A880024E023254D3B
:10318C00254F85F82230EC772C766C76AC7685F86A
:10319C0020406B6A43F4E0236B6285F82340FDF713
:1031AC0015FFFEF795F84FF0FF33AB62EB62FEF7BD
:1031BC001FFAFEF7B5F8194800F09CF90120FFF74B
:1031CC0025FF0220164DFFF721FF00F06DFB154B7C
:1031DC0015495D61154B4FF4806205930123284618
:1031EC00CDE90343CDE901443B46009400F042F99C
:1031FC0006466A7B284622F004026A7302F093FEAC
:10320C002046FFF77BFF3A4631462846FEF740F84A
:10321C00580C002000ED00E04930000010040020A4
:10322C0080030020E405002098150020FE760000A5
:10323C002DE9F341044617461E46EFF3118820236F
:10324C0083F31288BFF36F8FC368334A7BB18068F6
:10325C009168884219D057EA060318D188F311886F
:10326C00BFF36F8F6FF00F0002B0BDE8F081916873
:10327C0091F90E100133E36093682161A36088F328
:10328C001188BFF36F8F0020EEE72169F2E791F907
:10329C000E1090F90E306FF07E029942A8BF1946BD
:1032AC009142B8BF11468B422DDD02F0F4FD05466C
:1032BC0022464146CDE90076184800F0F3F9002883
:1032CC00E1D0EFF31186202383F31288BFF36F8FC5
:1032DC00A068D0B1236821699C420AD04BB193F904
:1032EC000E309942A8BF19466FF07E039942B8BFC1
:1032FC00194602F0D0FD40B13146084800F066FA9C
:10330C006FF00A00B0E70025D2E7002DF4D186F368
:10331C001188BFF36F8FF3E7E4050020500C0020F9
:10332C00F8B583680546002B40D0234A9268934237
:10333C003FD1C368012B03D9013BC3600020F8BD0A
:10334C00EFF31187202383F31288BFF36F8F01698A
:10335C00806802F0A0FD2C68A54207D10023C5E9C6
:10336C00023387F31188BFF36F8FE7E7002CF5D09A
:10337C00D4E90032002613605A60637BC4E900660E
:10338C0023F002036373A66004F1180002F068FED8
:10339C00AC6094F90E3020462B61C4F8886002F0C2
:1033AC00C2FD3946054800F011FAC7E76FF0150069
:1033BC00C5E74FF0FF30C2E7E4050020500C0020B9
:1033CC0070B5EFF31186202383F31288BFF36F8F50
:1033DC000468A0421BD0D4B1D4E90032002513609C
:1033EC005A60637BC4E9005523F002036373A56044
:1033FC0004F1180002F034FE2046C4F8885002F0A4
:10340C0092FD3146BDE87040064800F0DFB9D0E9C6
:10341C0002329A4218BF0133836086F31188BFF3DE
:10342C006F8F70BD500C002013B5EFF31181202469
:10343C0084F31288BFF36F8F846844B1013C8460BD
:10344C0081F31188BFF36F8F002002B010BD52EAD8
:10345C00030406D181F31188BFF36F8F6FF00F0057
:10346C00F3E7CDE900230246014800F01BF9ECE735
:10347C00500C00202DE9F043984685B000F158031C
:10348C00C0E91633109B002503730423073222F086
:10349C00070643730F9B01EB06090F4683734946DE
:1034AC00C0E906558560C5730446FDF781FB0E9B8C
:1034BC00073020F00700A067C4E91C7602930D9B2F
:1034CC00A9EB000901930C9B4A46009339464346ED
:1034DC002046FDF7C1FE064B65659B6884F86C5071
:1034EC0003B1DB6F4846E36705B0BDE8F08300BF6E
:1034FC00E405002040F2011383810023C0E91C3352
:10350C00C367014B98607047E40500206FF00A0117
:10351C00094A9368C3F888100849C3F884004B68BB
:10352C0043F080534B60002383F31188BFF36F8FFC
:10353C009368D3F888007047E405002000ED00E0A4
:10354C0070B590F90D20437B002A36DBD90634D1B7
:10355C001B4C63F07F032246437352F8183FE1691A
:10356C00934207D1C0E900210860E06111E0994263
:10357C00F8D01B68002BF5D090F90E5093F90E6023
:10358C00B542F4D0AE42F2DD5968C0E900310860B2
:10359C005860A569954200D005B9E568A3685A7BC7
:1035AC00D20604D1DA897F2A01D9AA6932B1AB4299
:1035BC0002D0284600F0FAFA656170BD6361FCE741
:1035CC00E405002038B590F90D200146002A437B14
:1035DC0004DA03F07F03437302F06BFC0D4D2A46B3
:1035EC0052F8184FAB68944200D004B9EC688B4287
:1035FC0007D05A7BD20604D1DA897F2A01D9A26975
:10360C002AB1A34202D0204600F0D0FA23466B61C7
:10361C0038BD00BFE4050020B3F1FF3F08BFB2F195
:10362C00FF3F03D00249183000F040BB704700BF89
:10363C00975F000038B5194CA168E0690B688142AE
:10364C0014BF1A46002249680B605960A368E169EF
:10365C002AB9134AC3E900210B60E3610CE093F92A
:10366C000E0092F90E50A84214D0854212DD51681A
:10367C00C3E900210B605360A569094B9D4200D042
:10368C0005B9E568A3689D4202D0284600F08EFA81
:10369C00656138BD9142DCD01268D9E7E4050020A1
:1036AC00FC050020F8B5DDE906670D4B0C46986863
:1036BC0011460C4A1060EFF31182202282F312881B
:1036CC00BFF36F8F9D68284602F005FC28463246F2
:1036DC003B46FFF7A1FF2046BDE8F840FFF716BFB9
:1036EC00E405002004060020F8B50446EFF311872A
:1036FC00202383F31288BFF36F8F437B49B203F00F
:10370C001F02002A0CBF0126002639D103F07F03CB
:10371C002D4D437302F0CDFB2A46437B817363F03E
:10372C007F03437352F8183F934227D1E869C4E9E9
:10373C0000200460EC610FE09842F8D01B68002B6D
:10374C00F5D093F90EC06145F6D08C45F4DD59687F
:10375C00C4E900310C605C60AC69944200D004B9DF
:10376C00EC68AB689C4202D0204600F01FFA6C61FA
:10377C0087F31188BFF36F8F3046F8BDE869DEE739
:10378C009B071ED5856802F094FB81732B689D42C4
:10379C0009D16B68C4E900531C606C60E8E76A6887
:1037AC009342F6D01B68002BF3D093F90E20914274
:1037BC00F5D08A42F3DD5A68C4E9003214605C60CB
:1037CC00D6E78173D4E700BFE405002049B9EFF3D5
:1037DC00058030B9054B5A699B689A4201D0FFF7B6
:1037EC0095BE81F31188BFF36F8F7047E4050020FD
:1037FC00034648B9EFF3058232B9064A516992681B
:10380C00914201D0FFF782BE83F31188BFF36F8F13
:10381C00704700BFE4050020EFF31181202383F3F0
:10382C001288BFF36F8F054B9A68D37B013BD37320
:10383C0081F31188BFF36F8F704700BFE405002040
:10384C0070B5EFF31186202383F31288BFF36F8FCB
:10385C00144DAB68DA7B0132DA732A4652F8184FF2
:10386C00944200D004B9EC685A7BD20604D1DA89B0
:10387C007F2A01D9A2692AB1A34202D0204600F0C6
:10388C0095F923466B6186F31188BFF36F8FEFF3C5
:10389C001180202383F31288BFF36F8FBDE8704033
:1038AC00FFF7A6BFE4050020024B03F11802C3E9A1
:1038BC0006227047E405002070B5EFF31186202333
:1038CC0083F31288BFF36F8F1B4CA168E0690B6800
:1038DC00814214BF1A46002249680B605960A368E4
:1038EC00E1692AB9154AC3E900210B60E3610CE0D8
:1038FC0093F90E0092F90E50A84218D0854216DDAD
:10390C005168C3E900210B605360A5690B4B9D42C4
:10391C0000D005B9E568A3689D4202D0284600F0A6
:10392C0045F965613046BDE87040FFF7EFBD8A424E
:10393C00D8D01268D5E700BFE4050020FC050020B4
:10394C00F8B550EA010306460C4603D1FFF7B4FF65
:10395C000020F8BDEFF31187202383F31288BFF307
:10396C006F8F124D124BA8681860FFF72BFEA868DA
:10397C00234632460F49183000F098F9AA680446DD
:10398C00537B384643F004035373FFF7BFFDAB681A
:10399C00D3E90A23B3F1004F08BF002AD8D102F0B3
:1039AC0087FB201A20EAE070D3E700BFE405002073
:1039BC0004060020975F000038B50446EFF311852C
:1039CC00202383F31288BFF36F8F437B5B070FD5E4
:1039DC00183002F045FB637B204623F0040363732D
:1039EC00FFF7AEFD2946BDE838400448FFF7EEBEB0
:1039FC0085F31188BFF36F8F38BD00BF500C0020CA
:103A0C00014B9868704700BFE40500202DE9F8438E
:103A1C000446077BEFF31185202383F31288BFF351
:103A2C006F8F437B190705D585F31188BFF36F8F13
:103A3C00BDE8F883D90943F008025DD14273A3684D
:103A4C0013B1204602F03DFA04F1180002F008FB15
:103A5C00A66D04F15808B04511D04FF0000976B1AD
:103A6C00304602F02EFA06F1180002F0F9FA304650
:103A7C00C6F88890FFF764FDA66DB045EFD1DFF86E
:103A8C00C080D8F808309C423ED1EFF30589B9F1DB
:103A9C00000918BF4FF00109D8F81860294A96425E
:103AAC0000D00EB9D8F80C60B34202D0304600F00A
:103ABC007DF82046C8F8146001F061FDB9F1000FE3
:103ACC0002D02148FFF716FDD8F808309C4231D1BE
:103ADC00EFF3058373BB227BD20718D42846FFF77C
:103AEC0015FDFB07A4D5002383F31188BFF36F8F5B
:103AFC000423184602DF9BE703F07F0343F008031F
:103B0C00437302F0D6F99AE74FF00009C4E785F346
:103B1C001188BFF36F8F83F31188BFF36F8F04236A
:103B2C00184602DFEFF31180202383F31288BFF3D2
:103B3C006F8FD4E785F31188BFF36F8FD1E700BF88
:103B4C00E4050020FC05002010040020427B034605
:103B5C0012F01F0210D10A4988420DD00949086899
:103B6C0068B1D9897F2909D893F90E20064B1B68B7
:103B7C009A42B8BF0020704700207047104670472B
:103B8C00F00200200C020020080600200122044B49
:103B9C00C01A044BC0105843034B1A54704700BF53
:103BAC00A0040020ABAAAAAA500C002070B50D4BA3
:103BBC000D4D1E7CFFF7CAFF06EB460305EBC30554
:103BCC000446284602F04CFA0022084B9A553CB1A8
:103BDC00621E2846BDE870400549D31700F066B850
:103BEC0070BD00BFE4050020A0040020500C002094
:103BFC00993B000038B5EFF31185202383F312882D
:103C0C00BFF36F8F0F4B104A9C681068A04206D10F
:103C1C00FFF7CCFF85F31188BFF36F8F38BD002100
:103C2C001B7C1160094AD35C002BF3D02046FFF7B4
:103C3C008DFF0028EED0637BDB0601D1FFF7FAFC89
:103C4C002046E5E7E405002004060020500C002087
:103C5C00024B1868984208BF0020704710020020E1
:103C6C00034B1B680BB9FEF7D5BA0020704700BF99
:103C7C000C06002030B570B10B4B5B6898420AD033
:103C8C00036843B1D3E90421D0E90445121941EB8F
:103C9C000501C3E90421D0E9003213605A60002306
:103CAC00C0E9003330BD00BF10020020B3F1FF3F6C
:103CBC0008BFB2F1FF3F2DE9F84F0446994615466F
:103CCC001F467AD08160EFF31188202383F312888A
:103CDC00BFF36F8FB9F1000FDFF8E4A020DBFFF723
:103CEC00BFFFDAE90027013549F100092D1849EB2E
:103CFC00E07306464FF00109C4E90453AD1843EBD9
:103D0C000707FFF7A5FF0346DFF8B8E0DEF804A0CD
:103D1C00EBB9C4E900EACAF80040CEF8044028E048
:103D2C006FF00103DAE900125B1A4FF0FF3161EB1F
:103D3C0002025B1B62EB0902012B72F10001BCBF9A
:103D4C00012300224FF00009C0E90432D9E7D3E97E
:103D5C00041CD4E904208A4270EB0C0B24DA891A77
:103D6C005A686CEB0000C3E90410C4E9003214601B
:103D7C005C60FFF76DFF84420ED1134B1B685BB97F
:103D8C00B9F1000F02D1FFF76BFF0646304602F087
:103D9C0050F90021FEF752FA88F31188BFF36F8FA8
:103DAC0028463946BDE8F88F521A60EB0C009A454C
:103DBC00C4E90420ADD01B68AAE700252F46EFE725
:103DCC00B8040020100200200C0600202DE9F0475A
:103DDC00EFF31185202383F31288BFF36F8FDFF885
:103DEC00A0900026C9F800000027FFF731FFDFF88C
:103DFC009480D9F80030D8E900ECD91750B1D0E94B
:103E0C000442A34271EB020A1BDAE41A62EB0102D0
:103E1C00C0E90442002413EB0E034CEB01012046D5
:103E2C00C8E90031C9F8004002F003F92146FEF759
:103E3C0005FA85F31188BFF36F8FBDE8F047FFF7E4
:103E4C00D9BE14EB0E024CEBE473C0E90467C8E96D
:103E5C000023FFF70FFF85F31188BFF36F8F836883
:103E6C009847EFF31185202383F31288BFF36F8FEC
:103E7C00D9F800301B1BC9F80030FFF7E9FEB8E792
:103E8C000C060020B804002010B5EFF31184202399
:103E9C0083F31288BFF36F8FFFF7E2FE0346054AE8
:103EAC00D2E90001181841EBE37184F31188BFF3D8
:103EBC006F8F10BDB8040020F8B50D4E0D4C0E4D93
:103ECC0033680E48984767782B680C4898473368D6
:103EDC000B489847022F08D12478E31F5C425C41C1
:103EEC002B68074898472046F8BD0024F8E700BF28
:103EFC003C02002010060020380200209C0200200A
:103F0C008802002070B51D4E1D4C33681D48984723
:103F1C002378590744BF23F00403237023789A07AE
:103F2C0005D500F0C1F8237823F002032370164D59
:103F3C0014482B689847336814489847637813B132
:103F4C00134802F0E7F8002304211148637000F0D5
:103F5C00CBF82B680D48984733680A489847237864
:103F6C00DB0705D502F0D3F8237823F00103237087
:103F7C002B680448BDE87040184700BF3C02002085
:103F8C001006002088020020380200209C0200202D
:103F9C00140600202DE9F041FFF78EFF18B1002424
:103FAC002046BDE8F081364F36483B6898470446BA
:103FBC0020B16FF08F04FFF7A5FFF1E7324D2B789E
:103FCC00D80706D402F0A1F804462B7843F001037D
:103FDC002B702E4E2B483368984710B1002CE8D02C
:103FEC00E9E7002CE7D13B682648984704460028AF
:103FFC00DFD12B78990706D400F04EF804462B78C5
:10400C0043F002032B7033681E4898470028E5D113
:10401C00002CD0D13B681B4898470028C9D1336885
:10402C00184895F8008098470028C2D13B6818487A
:10403C00984704460028BCD16B7843B918F0010F9F
:10404C0005D0144802F064F8022304466B70336800
:10405C000F4898470028C1D1002CACD13B680948C7
:10406C0098470028A5D12B7806485A075CBF43F027
:10407C0004032B7033689847002890D099E700BF51
:10408C003C0200208802002010060020380200208C
:10409C009C020020140600200122024B002083F811
:1040AC0080257047180600202DE9F0410A4C0025A8
:1040BC0026464FF0010803272046C4F820802777B6
:1040CC00013502F005F8202D04F12C04F4D1002365
:1040DC0086F88035BDE8F08118060020014B1B687E
:1040EC00184700BF1802002010B50A46044619B143
:1040FC00024B00211B68984710BD00BF1C0200201A
:10410C0010B50C4C206802F0B4F90B4A1368591C1A
:10411C0011604BB9094A4820D2F8003443F0070328
:10412C00C2F80034FDF730F82068BDE8104002F00A
:10413C00A6B900BF240200209C0B00200080045074
:10414C0038B5164D286802F094F9154B1C68013CE3
:10415C001C60ECB94820FDF725F80722114BC3F879
:10416C000823D3F8002422F00702C3F80024C3F874
:10417C000041D3F80021C3F80441D3F804214FF4D3
:10418C008072C3F80841D3F80831074BC3F8882173
:10419C002868BDE8384002F072B900BF2402002044
:1041AC009C0B00200080045000E100E070B5104D25
:1041BC00104E2B68B3420DD0FFF7A2FF00F0D8FCD5
:1041CC0000F014FD40B101F0B2FF0446FFF7B8FF58
:1041DC0044B92E60002405E000F0D2FA044618B170
:1041EC00FFF7AEFF204670BD02F0A4F8EDE700BF6C
:1041FC0020020020117365000022074BC3F8102128
:10420C00C3F80C21C3F80021C3F80421C3F808211A
:10421C00C3F81421704700BF0050045008B5FFF7D5
:10422C00EBFF01230360104B0A6832B9D3F80C2161
:10423C001AB9D3F80821002AF6D00B687BB90B4BBE
:10424C0099420ED0A3F58473D3F80831002B0CBF20
:10425C004FF0FF306FF00200FFF7CEFF08BD0020DB
:10426C00FAE74FF0FF30F7E70050045008510450C4
:10427C0038B505460C4691B10021012001F0CBFD6B
:10428C0008480949C0F80055C0F80445FFF7C6FFB7
:10429C0000210446084601F0BEFD204638BD6FF0F3
:1042AC000104FAE70050045000510450034B044938
:1042BC00C3F800050348FFF7B1BF00BF005004501E
:1042CC00045104500450045010B504460021012040
:1042DC0001F0A1FD064B0749C3F800450648FFF75E
:1042EC009DFF00210446084601F095FD204610BDB7
:1042FC0000500450085104500850045038B50C4676
:10430C0059B1074D0749C5F800050748FFF786FF67
:10431C0010B9D5F80835236038BD6FF00100FBE704
:10432C0000500450105104500C5004502DE9F0472B
:10433C00804600244FF010091E4E94B00DF1270555
:10434C0025F01F0506F1200A012210211A4801F060
:10435C0059FF2B1900935246102320211548CDF8F4
:10436C00049000F04BFA0746F8B9D6E90C32103439
:10437C00013342F10002302CC6E90C32E4D1B8F121
:10438C00000F04D022464146284601F02EFF2E464F
:10439C00084C0FCE0FC496E80F00203584E80F00B0
:1043AC0095E80F00103484E80F00384614B0BDE8CF
:1043BC00F08700BFC0040020E0040020F0B5194DC8
:1043CC00194FAB6B8DB0BB4229D0184E306802F040
:1043DC0050F8402300221946284601F01DFF3021D9
:1043EC00684601F03AFF044678B96846FFF79EFF2D
:1043FC00044690B9302302461946684601F00CFF7A
:10440C0001220023C5E90C23AF63306802F037F8B2
:10441C00204601F08CFE0DB0F0BD0E24F5E7002017
:10442C00F9E700BFC0040020B4A5B4A52802002001
:10443C002DE9F04F99B00DF1570802F10F098246A2
:10444C000E46144628F01F084FEA191922B100290C
:10445C0067D0B2F5803F64D8334F344D386802F0E2
:10446C0008F8D5E90C3213430BD15046FFF7A6FFE1
:10447C00834630B1386802F002F8584619B0BDE8EE
:10448C00F08FD5E90C2319EB020243F10003B3F5CD
:10449C00803F14D3302102A801F0DFFEB8B902A886
:1044AC00FFF744FF83460028E4D130230246194627
:1044BC0002A801F0B1FE00220023C5E90C23DFF8AD
:1044CC0070A03CB92046FFF731FF8346D2E76FF06E
:1044DC00920BCFE7102C4FF001024FF01001504619
:1044EC00A14628BF4FF0100901F08CFE1023524654
:1044FC002021CDE900830D4800F080F98346002887
:10450C00B8D14A463046414602F041F8D5E90C3262
:10451C00013342F10002C5E90C32A4EB09044E440C
:10452C00CFE76FF0860BA8E728020020C00400201C
:10453C00E00400202DE9F04F89B007460C461546E3
:10454C001E4601F0D4FE78B97B690090C3F30132AA
:10455C0062F305108DF8000010F0300007D1B96837
:10456C0089070FD06FF0860009B0BDE8F08F1028D6
:10457C0008D1BDF8023023F4F87343F4A873ADF8F6
:10458C00023053E0DBB2F82B02D06FF08500EBE782
:10459C0000234FF0010B984619469C46D7F808E0CB
:1045AC00DFF8CC9159F804AB1EEA0A0F08D00BFACD
:1045BC000CF343EA080303F07F08012341EA0A01E4
:1045CC000CF1010CBCF1070FECD12BB19DF80330B1
:1045DC0068F347038DF803303EEA0101D5D17B889F
:1045EC00FF2B35D005D8802B34D0C02BCDD1022356
:1045FC0006E0B3F5807F2FD0B3F5C07FC5D106237D
:10460C009DF8021063F306118DF8021010B91EF01C
:10461C00030FA7D13B79022B2BD01FD8012BA1D193
:10462C00BDF8021063F3C811ADF80210012A39D09D
:10463C00032A23D0002A95D13B88B3F5105FA4D16F
:10464C00182E03D0202E01D0102E8BD1494F2DE0E7
:10465C000323D5E70123D3E70423D1E7032B02D0AF
:10466C00FF2B7FF47FAF0221BDF8023061F3C8133A
:10467C0085E7BDF8023043F4C07380E7412E0ED0BD
:10468C00202E05D006D8102E02D0182E7FF46AAF3B
:10469C00394F0BE0302EFBD0612E7FF463AF013528
:1046AC00013EF5E7302E7FF45DAF344F4FF000083C
:1046BC000F364FEA1619C14515D11F2E1CD81C22D6
:1046CC00002101A801F070FF4FF0000A4FF0FF39F4
:1046DC00D04518D11F2E04D9BA20FFF7F5FD0028BC
:1046EC0035D1002040E704EB080001F0ACFD0028B8
:1046FC003AD008F10108DEE74146204601F0DFFD23
:10470C000028DCD030E707EB0A124FEA0A130692B6
:10471C00BAF1000F1ED1009A0792BDF802202B446B
:10472C00C2F3C11205920DF1040C03F1100E624696
:10473C0018685968083303C273459446F7D101A928
:10474C0004EB0A00FFF794FD38B101F0D0FD6FF0D7
:10475C00920009E7CDF81C90DFE71C2101A801F0BD
:10476C0066FD0AF1010AB3E76FF08A00FCE600BFB0
:10477C00CC710000400081510000002010840450D6
:10478C0010B590B01C22002101A801F00DFFF820FB
:10479C0001F059FD08B3202200200DEB0201FFF7B8
:1047AC0047FE0446F8B901A84FF4807101F07DFD75
:1047BC000E4B0F4904930F4BCDE901130E4BF8210F
:1047CC00069320230DEB0302FFF7B4FE20210446D1
:1047DC000DEB010001F02BFD05E0F92001F033FD9C
:1047EC000028D8D10446204610B010BD0010C004DB
:1047FC0000240001014B4E80F800FF7F2DE9F341AE
:10480C001D464FF48073284C8046002017460E46F8
:10481C00019300F037F901AB23601123234A0121E6
:10482C00C4E9022304F11003636040F61103E36151
:10483C0004F1200363612123089AE3621C4B46F0C8
:10484C0000561A60099A45F0005542F00052C3E92F
:10485C0001122022C4F81080A6612762A562616251
:10486C00DA60BFF35F8F4FF0A3421460BFF35F8F2A
:10487C00BFF35F8F1361BFF35F8FBFF35F8F0323B2
:10488C005363BFF35F8FBFF35F8F9363BFF35F8F90
:10489C0001F08CFD431C0446FAD0002000F01CF9FA
:1048AC00204602B0BDE8F081B00B002004000020CF
:1048BC00A00B0020BFF35F8F094A1368BFF35F8F13
:1048CC0043F48071BFF35F8F1160BFF35F8F23F4EC
:1048DC008073BFF35F8F1360BFF35F8F704700BFB0
:1048EC000010805108B5FFF7E5FFBFF35F8F064A54
:1048FC001368BFF35F8F43F00103BFF35F8F136047
:10490C00BFF35F8F08BD00BF0010805170B500264B
:10491C00C0E9006605460C46FFF7F2FB01232B703D
:10492C00FFF7C8FFBFF35F8F204BDB68BFF35F8FD0
:10493C009B08013BACB3226842B19A4205D9FFF700
:10494C00FFFB6FF03F002E7070BD1346D4E90115CC
:10495C00E068002908BF4FF40071002808BFF1205F
:10496C002469BFF35F8F114A9360BFF35F8FBFF36E
:10497C005F8F1564BFF35F8FBFF35F8F5064BFF31E
:10498C005F8FBFF35F8F5163BFF35F8F44F480245D
:10499C0044F00104BFF35F8F1460BFF35F8F0020FE
:1049AC00D2E74FF40071F1202546DAE70010805170
:1049BC0070B503780D461446002B53D0BFF35F8FB0
:1049CC002D4A136BBFF35F8F5908C3F34203052BBA
:1049DC004BD011F0060F02D14FF0FF3070BD436881
:1049EC00D3B9BFF35F8F5368BFF35F8F032BF3D93A
:1049FC00224B2349BFF35F8FD2F88060BFF35F8FE8
:104A0C00BFF35F8F43F8046BBFF35F8F8B42F1D121
:104A1C00FFF768FF01234360BFF35F8F164B9A6863
:104A2C00BFF35F8F0132B4EB021F21D8BFF35F8F4E
:104A3C005A68BFF35F8FB4EB820FCDD884B1BFF34C
:104A4C005F8FD3F88020BFF35F8F291D05F8012BF2
:104A5C008D424FEA122204F1FF34EFD0002CF5D135
:104A6C000020BBE76FF02000B8E76FF05100B5E70E
:104A7C006FF03F00B2E700BF001080511010805162
:104A8C002010805110B50446FFF73AFB104B186804
:104A9C0001F0EFFC0CB101232370BFF35F8F4FF0DB
:104AAC00A3430022DA61BFF35F8FBFF35F8F4FF038
:104ABC00FF321A63BFF35F8FBFF35F8F3422DA616B
:104ACC00BFF35F8F0122034BC3F8042310BD00BF5B
:104ADC002C0200200080045010B5044638B9FFF7B2
:104AEC002FFBBDE81040074B186801F0C8BC0378D9
:104AFC003BB1FFF725FB034B186801F0C0FC00230A
:104B0C00237010BD2C02002038B5164CD4F800517F
:104B1C00C5B1BFF35F8F4FF0A343996ABFF35F8FAB
:104B2C00BFF35F8F4FF0FF321A63BFF35F8F002329
:104B3C00C4F80031D4F800310B4B1868BDE838408C
:104B4C0001F0B0BCD4F8083153B100F06BF801F0AF
:104B5C005EFCC4F80851D4F808310121034BECE792
:104B6C0038BD00BF00800450340200203002002009
:104B7C0008B5074B186801F084FC064B186801F067
:104B8C0080FCBDE80840002248201146FCF72CBBF5
:104B9C00340200203002002038B5094B1C7864B177
:104BAC00084B4FF0FF311D68284601F06CFC4FF0AC
:104BBC00FF310446284601F073FC204638BD00BF87
:104BCC004F0C00203402002010B5064CE36C3BB9AE
:104BDC00214651F84C3B986901F01DFC0123E3641C
:104BEC00014810BDE00B00202C0C002010B50B4B25
:104BFC000B4C236003F5C04363602461FFF7E4FFB3
:104C0C0050B1236D0020B3F5007FCCBF4FF480630F
:104C1C004FF40073A36010BD0E20FCE70020805100
:104C2C00E00B002000487047E00B00202DE9F0431A
:104C3C004FF0000985B00546CDF8049000F10C0743
:104C4C00EFF31188202383F31288BFF36F8F8368EF
:104C5C00594003EA02060A4053400E4901AACDE925
:104C6C00023901F0C4F9019C3CB12046C4F888908B
:104C7C000021246E01F066F9F6E7DDE9023223EA41
:104C8C00020338464146AB60FEF7A0FD304605B046
:104C9C00BDE8F0833F6500000FB407B504AA064BCE
:104CAC0052F8041B1868019200F008F803B05DF884
:104CBC0004EB04B0704700BFD47000002DE9F04F36
:104CCC0043688DB015468046029383789A0740F16D
:104CDC000D8100240E78002E00F00A81252E0BD0B9
:104CEC004B1C0393013441463046029B98470028E5
:104CFC00C0F2F6800399EDE74E788B1C252E0393BA
:104D0C00F0D00027B946BB46BBF11F0F38D8A6F12F
:104D1C002003102B0AD8DFE803F02A09093009090F
:104D2C00092109090928092D09091F00A6F13003D9
:104D3C00092B33D92A2E37D11BF0400F55F8043BE1
:104D4C0040F08280002BA7BF4BF0200B9946C3F19B
:104D5C0000094BF0280B01E04BF0010B039B13F8FF
:104D6C00016B0393002ECFD130E04BF0020B4BF0D4
:104D7C00040BF3E74BF0080BF0E74BF0100BEDE7EF
:104D8C00BBF17F0F19D8A6F13003092BD2D81BF039
:104D9C00400F03D00A2101FB0737DFE70A214BF054
:104DAC00200B01FB0939D9E72E2E06D11BF0400F41
:104DBC0040F09E804BF0400BD0E76C2E31D02BD8BE
:104DCC00682E36D06A2E3CD04C2E3AD0002F46F0AE
:104DDC002003B8BF2BF04002A3F16501BCBF002734
:104DEC001FFA82FB022901D9612B2FD10735072726
:104DFC00DFF8ACA225F0070508351BF0080F66D0CC
:104E0C000AEB070B56465E4563D1A4EB0A0AA9EBE5
:104E1C00070906EB0A026FE1742E9FD07A2E9DD003
:104E2C00D4E71BF0800F18BF4BF4007B4BF0800BCA
:104E3C0094E71BF4807F18BF4BF4007B4BF4807B12
:104E4C008CE74BF4207B89E71F4687E7A6F16301CB
:104E5C00122900F2F080DFE811F013004F00EE0091
:104E6C00EE00EE00EE004F00EE00EE00EE00EE0065
:104E7C00EE00FE00E900EE00EE001B00EE00AF00BD
:104E8C0055F8043B01270DF1180A8DF81830B4E7DA
:104E9C0055F804AB834BBAF1000F08BF9A461BF0D0
:104EAC00400F504614BF39464FF0FF3101F084FBE0
:104EBC000746A2E741462020029B984700280FDBBB
:104ECC00013EB742F6D34C44B146A41B98E74E467C
:104EDC00F7E7414616F8010B029B9847002892DA37
:104EEC0098F8023043F0040388F802304FF0FF3496
:104EFC0020460DB0BDE8F08F1BF0800F34D01BF4B2
:104F0C00007F2CD0073525F00705AA4669685AF8AA
:104F1C00080B2BF010050029ADB237DA404245F4EE
:104F2C00806561EB41010DF1180B0A235A4601F023
:104F3C004FFBA0EB0B0301936B0662D5019B25F095
:104F4C0001019F4289B240F3A180002E00F09980AC
:104F5C0015F0100240F09C80BB460D4623E0AA469B
:104F6C005AF8040BC117D4E7AA461BF4807F5AF8F1
:104F7C00041B01D10846F5E71BF4007F19BF48B2AA
:104F8C0041F3C01108B241F3C031C2E750EA01034A
:104F9C00C9D11BF0400FC6D0002FC4D12BF0110289
:104FAC00BB46019795B240F2064115EA01021CBFBF
:104FBC000BF1010B00222CE02BF010020A231FFA3C
:104FCC0082FB1BF0800C49D01BF4007115BF073518
:104FDC00AA4625F007055AF8040B1EBFAA466968B5
:104FEC005AF8080B50EA010545D12BF016051BF0B9
:104FFC00400FADB242D0002F40D12BF017020197D9
:10500C0095B215F0100248D0019B002E42D103F14D
:10501C00010B29075AD4EB0706D5D9456FDDA9EB4F
:10502C000B030199CB465F185B4649E04BF0100B24
:10503C0010237826C5E7782B04D1C6F1780343F00A
:10504C001003BEE741462520029B98470028FFF637
:10505C0047AF023447E608230026B2E7AA461BF402
:10506C0080715AF8040BBDD01BF400711ABFC0B28A
:10507C00614680B2B6E72BF0060295B20DF1180B23
:10508C0054E725F01105BB46ADB28CE70D46B8E7E9
:10509C003B460D4603F1020BBBE7DDF804B082E79B
:1050AC000A77000003770000CDE904324146202046
:1050BC00029B98470028FFF613AF049B059A013317
:1050CC009945F1DCA4EB0B019B46CC180AB3414685
:1050DC003020029B98470028FFF602AF8EB90134AE
:1050EC002744391B019B994224DC1D4655BB019A70
:1050FC00A9EB0B09554622441446914433E0019F19
:10510C0092E7023441463046029B98470028E7DA82
:10511C00E6E640F206410D42E2D015F0020F04F132
:10512C000104414614BF2B20202015F4806F18BFBA
:10513C002D20E9E741463020029B01349847002896
:10514C00CFDACDE606AB013D4146585D029B984750
:10515C000028CBDAC4E641462020029B0134984754
:10516C000028FFF6BDAEA9EB0403002BF3DCC1E570
:10517C00704703460A46F0B41979DB88006813437C
:10518C00DC028768066906D513F4402F03D0DA07D2
:10519C0048BF83F44023012534688D4023F48012EA
:1051AC00DB074CBF2C43AC4334603B68F0BC184766
:1051BC00034601211B790068994083685B69184795
:1051CC00836800EBC101B3F5004F2CBF51F82200EE
:1051DC0031F81200704700EBC1018068B0F5004F48
:1051EC002CBF41F8223021F812307047012208B54B
:1051FC00FFF7E6FFD04008BD836800EBC101B3F5B3
:10520C00004F08D34B681AB143F001034B60704751
:10521C0023F00103FAE74B881AB143F001034B80EA
:10522C00704723F00103FAE753000122FFF7D3BFC5
:10523C008368481CB3F5004F34BF0423082308339C
:10524C00A0EBD300B0FA80F0C0F11F0070472DE93D
:10525C00F0410D4686680446FFF7C8FFB6F5004FCF
:10526C00014601D3012832D02046FFF7E1FF04EBC1
:10527C0080010E6996B90122E36882401343E36012
:10528C0002220D612B4629462046FFF7A4FF03227C
:10529C0029462046BDE8F041FFF79DBF022231466A
:1052AC002046FFF78DFF0746034629462046FFF7A9
:1052BC0092FF0322334629462046FFF78CFF3946DE
:1052CC002B462046FFF787FF02223146E1E7BDE877
:1052DC00F081B2F5802F2CBF082304232DE9F04177
:1052EC000026D21A8C18CD1D25F0070524F00704D2
:1052FC00641BE408056021462846AC60EE60FFF7AD
:10530C0097FF421D9200013002F107074FEAD707C1
:10531C003146A2F1100205F11000B8BF324601F07F
:10532C0043F93A4631462846FFF77EFF334632466C
:10533C0031462846FFF74FFFA4EB070828463146B5
:10534C000122FFF759FF42463946FFF76DFF3B46F6
:10535C00324639462846FFF73EFF21462846FFF7DE
:10536C0063FF4346324621462846FFF734FF214669
:10537C0028460122FFF740FF3946BDE8F041FFF710
:10538C0066BF002070470FB407B504A951F8040B91
:10539C000191FBF75DFA03B05DF804EB04B07047C4
:1053AC00038B13F0070305D10368002B0CBF0020FF
:1053BC0003207047022B05D1408BB0FA80F04009D6
:1053CC0080007047012B05D10368002B0CBF002017
:1053DC00052070470020704710B50C4600B111B97C
:1053EC006FF0150010BD081D00F093F80028F9D1DE
:1053FC00A368032BF6D9F3E72DE9F0410D460746D8
:10540C001946281D90461E4600F094F8044638B103
:10541C003346424629463846A446BDE8F04160472B
:10542C00BDE8F08110B4EFF31182202484F31288CC
:10543C00BFF36F8F416110BC0121FBF73BBA38B54C
:10544C000C46054658B151B10B6843B14B6833B1AA
:10545C001C22002101F0A8F800202C6138BD6FF04F
:10546C001500FBE770B505460E46FFF7B5FF041EA9
:10547C0014DBEFF31182202383F31288BFF36F8FB9
:10548C004FF6FF716B8B2C8B8B4204F0070407D10A
:10549C0082F31188BFF36F8F6FF00A04204670BD42
:1054AC00022C0CD101336B8382F31188BFF36F8F05
:1054BC000023224631462846FFF79EFFEEE7062CD6
:1054CC0014D8DFE804F004131313041A04000023A7
:1054DC0033606B683BB9C5E90066ACB9022128465C
:1054EC00FBF7E8F9DAE71E606E60F6E782F31188E5
:1054FC00BFF36F8F6FF00404D0E782F31188BFF312
:10550C006F8F6FF08504C9E782F31188BFF36F8F3B
:10551C00C4E7034658B1426802F00302012A03D0E3
:10552C00032A04D1026812B10020986070476FF012
:10553C00150070474268034602F00302032A4FF03D
:10554C000002816014BF104600685A6070477047B3
:10555C0001F02AB801F01BB801460068FBF7F4BA59
:10556C0008B5FBF721FBBDE80840FBF741BB002168
:10557C000120FBF7E9BA036F83F30B8870476FF0D8
:10558C008500704761B662B680F31188BFF36F8FE8
:10559C00704772B6002383F31188BFF36F8FBFF38C
:1055AC004F8F30BF62B6BFF36F8F704772B6002358
:1055BC0083F31188BFF36F8FBFF34F8F20BF80F33E
:1055CC001188BFF36F8F62B6704740E800F313F495
:1055DC00803FD8B208BF6FF01500704730B50C682B
:1055EC004B6885B00A894D890094013B24F01F0457
:1055FC00234402F01F0242EA451223F01F036946BE
:10560C008DF808200393FBF7C1FE05B030BD08B53B
:10561C00FCF79EF8002008BD0C220369C9B201FBFF
:10562C000233186C00F00700704770B5C9B20369FB
:10563C00EFF31185202484F31288BFF36F8F0C26AF
:10564C0006FB0134246C14F0C00408D0A24206D02E
:10565C0085F31188BFF36F8F4FF0FF3070BD0122BF
:10566C0006FB01331A6485F31188BFF36F8F43680F
:10567C0003EBC1035B6898470020EFE78022FFF73C
:10568C00D4BFF8B5069F0469C9B2EFF31186202583
:10569C0085F31288BFF36F8F0C2505FB0144256C35
:1056AC0005F0070CBCF1010F0CD1276486F31188AF
:1056BC00BFF36F8FC4E90E23436853F8313098471A
:1056CC000020F8BD05F0C005AF4286F31188BFF38A
:1056DC006F8F0CBF6FF077004FF0FF30F1E713B511
:1056EC0080240094FFF7CDFF02B010BD10B41C2431
:1056FC000069CBB203FB0400002110BC104710461C
:10570C00FDF75EBE00F04DB9FCF710BF43680020FA
:10571C005B68DB680B607047436802EA01005B68FA
:10572C0021EA02015860002099607047436800200C
:10573C005B6859607047436800205B6899607047EC
:10574C0043685A68136821EA03000B40506000203C
:10575C009360704710B503695868F8B1884219D145
:10576C009C680868A142586000D1986000200860CD
:10577C002AB15A680A609A68596002B99960002087
:10578C0010E0814206D10868206098688142EDD112
:10579C009C60EBE7044600680028F2D1002AE8D1AF
:1057AC006FF0150010BDFDF72FB930B543681360CD
:1057BC00057A446804EBC504A34202D36FF00100E0
:1057CC0030BD5C798C4201D00833F0E70020F7E75C
:1057DC0043681B68D3F83031704743681B68D3F8B3
:1057EC008004C3F88004704742681368D3F84C01F6
:1057FC0050B10020926A12780A70C3F84C01D3F8A9
:10580C004C2101229A6270474FF0FF30704713B55C
:10581C0001AA0446FFF7C9FF002805DB019B22689B
:10582C0019791868FCF776FB02B010BD38B505463F
:10583C0000220121C620FBF7D7FCC620FBF7A4FCF5
:10584C006C680121E068FFF7E2FF6B681968636917
:10585C00C1F82435E28BA38BA07E1343228C134317
:10586C00628C1343627E9BB20243207E024313433D
:10587C00C1F86C3569680B68D3F8002242F48022B9
:10588C00C3F800220822C3F800254A6A0121C3F894
:10589C003C270022C3F840271965D3F830110029A2
:1058AC00FBD0C3F800256D680021E8682C68FFF771
:1058BC00AEFF0823C4F800352A7A52B9AB6AC4F893
:1058CC0004370123C4F80837C4F84C21D4F84C2110
:1058DC00A362002038BD08B50220FCF7D9F80020DF
:1058EC0008BD08B5FEF756FB48B1002383F31188B9
:1058FC00BFF36F8F0423184602DF6FF0040008BD5E
:10590C0003460020184700F089BA024610B511680A
:10591C0091B1B1FA81F3C3F11F000123834021EA55
:10592C000303D2E8EF4F8C4204D1C2E8EC3FBCF148
:10593C00000FF6D1EBD110BD6FF00B00FBE710B5EB
:10594C000368CB40DB0710D401238B40026843EA89
:10595C000201D0E8EF4F944204D1C0E8EC1FBCF137
:10596C00000FF6D1F2D1002010BD6FF01500FBE74F
:10597C00FCF778BD10B1012802D07047FCF7D6BDFA
:10598C00FCF784BE18B1012803D100F00CB800F06C
:10599C0008B8704708B5FCF7ADFEBDE80840FCF749
:1059AC0005BEFCF797BDFCF739BEF7B51646DDE929
:1059BC000847019001A81D46FCF7D6FE019BB6F1E5
:1059CC00000C18BF4FF0010C00EB83000B1E18BF2E
:1059DC000123002D43EA4C0314BF4FF00C0C4FF085
:1059EC00000C002C43EA0C0314BF4FF4706C4FF006
:1059FC00000C002F43EA0C0314BF4FF4403C4FF053
:105A0C00000CD0F8802043EA0C0322EA030301B116
:105A1C0009780EB13678760019430DB12D78AD00AA
:105A2C0031430CB12478240229430FB13F783F0451
:105A3C000C433C43C0F8804003B0F0BD1FB50DF1E2
:105A4C000F03019300238DF80F101A46194600938B
:105A5C00FFF7ABFF05B05DF804FB10B50446084634
:105A6C00FCF792FE04EB4004A08AC0F3401010BD7A
:105A7C0010B504460846FCF787FE04EB4004A08AE8
:105A8C00C0F3400010BD10B504460846FCF77CFE80
:105A9C0004EB4004A08A400B10BD70B504460846C8
:105AAC001646FCF771FE083034F810300D46DA0556
:105ABC0009D5C3F3432304EBC3023146284654F8FB
:105ACC00333052689847A3682BB131462846E268B8
:105ADC00BDE87040184770BD10B504460846FCF789
:105AEC0053FE00B204EB4000838ADA051DD5C3F3E4
:105AFC00432123F4F853838204F1120204F1580079
:105B0C0032F8023F13F4807F03D0C3F3432399424E
:105B1C000BD08242F4D1002204EBC1035A6004F191
:105B2C006000BDE81040FFF70ABF10BDF0B5044699
:105B3C00002001270546844695420AD1D4F8443109
:105B4C0033B10023C4F84431D4F8443140F400306C
:105B5C00F0BDEBB29B0003F580769B0807FA03F3CC
:105B6C00194208D054F806E0BEF1000F03D044F8F7
:105B7C0006C0A65918430135DEE738B504460D4674
:105B8C00FFF76BFFB0B12046FFF772FF90B92046CC
:105B9C00FFF779FF012322688340C2F8183323688A
:105BAC0000B203EB8003D3F8102522F00302C3F8F4
:105BBC00102538BD2846BDE838400021FFF73EBF10
:105BCC002DE9F0431746044685B00846FCF7DCFD8A
:105BDC00D7F800800E460546B8F1000F1FD02046BE
:105BEC00FFF746FF18B12046FFF737FF30BB002305
:105BFC000DF10F02CDE900338DF80E308DF80F301A
:105C0C00304643460DF10E01FFF7CFFE2AB204EBEE
:105C1C004202938A23F0020343F0010393827B68D0
:105C2C00002B34D03146204693F80080D3F80490F2
:105C3C00FFF71EFF28B1B9F1000F1FD06FF0150050
:105C4C0028E028B204EB4000838A23F4604323F05D
:105C5C0020038382B9F1000F10D0B8F1030FEDD8F7
:105C6C007B6821685B6893F800C001EB8C01B8F18C
:105C7C00000F12D1C1F81085C1F810852AB204EBBF
:105C8C004202938A23F01C0343EA88039382BB6885
:105C9C0053BB002005B0BDE8F083D1F8102522F0ED
:105CAC000302C1F81025226802EB8C03D3F81025EF
:105CBC0022F4473222F47C72C3F8102541F6F072BC
:105CCC00D3F8101502EA061242EA08420A43C3F856
:105CDC00102504EB4C03A3F86460838A43EA4C332D
:105CEC0043F020038382C9E73146D3E9007820468C
:105CFC00FFF7F2FE002FCCD063689F4206D004F170
:105D0C006000FFF702FE002804DAC3E7A368984599
:105D1C00F5D1002004EBC003C3E901782DB204EBEC
:105D2C004505AB8AC0B243EA402343F48073AB828F
:105D3C00AFE7C0E90312704770B504461546FFF78C
:105D4C008CFE48B10846FCF71FFD04EB4004002014
:105D5C00A38A5B0B2B7070BD6FF01500FBE790F8FE
:105D6C007400003818BF01207047FCF743BD2DE9C3
:105D7C00F34104461746FFF770FE0D46266800B344
:105D8C002046FFF775FE8046D8B92046FFF77BFE0C
:105D9C0005B2AD0005F5807246F802802168B25854
:105DAC002944D1F8102542F00102C1F810252FB179
:105DBC000122216802FA00F3C1F8143302B0BDE8E5
:105DCC00F081D6F8143328469B035CBF4FF40033A4
:105DDC00C6F81433FCF7D8FC04EB4004A38AC3F3D5
:105DEC008203042B11D0052B11D001A80195FCF7CF
:105DFC00BBFC019BC168D94001F00101023128466E
:105E0C0002B0BDE8F041FFF719BE0321F7E702210C
:105E1C00F5E7FFF7B2BEC9B2FDF7D4B808B1FBF78E
:105E2C0011BD704710B5436904463BB90020E268C8
:105E3C004042537843F00103537010BD984700283B
:105E4C00F4D00028B8BF4042FF28A8BFFF20E36869
:105E5C001870ECE740B1C368587810F001001EBF11
:105E6C001878B0FA80F040097047EFF311832023C3
:105E7C0083F31288BFF36F8FFEE708B5FFF7F5FFCA
:105E8C00202408B5EFF3118384F31288BFF36F8FCE
:105E9C00FFF77FFBF6E790F90E308B4201D0FDF750
:105EAC0023BC00207047EFF30580003818BF012099
:105EBC007047D0E9003213605A600023C0E9003308
:105ECC00704708B5FFF7F5FF437B23F002034373DC
:105EDC000023836008BD38B504460D46FDF772FB00
:105EEC00637B43F002036373E5B1A5602B689D42AD
:105EFC0009D16B68C4E900531C606C6012E06A68DD
:105F0C009A42F6D01B68002BF3D094F90E2093F92B
:105F1C000E108A42F3D09142F1DD5A68C4E9003286
:105F2C0014605C6038BD10B5EFF31184202383F34B
:105F3C001288BFF36F8FFDF703FB84F31188BFF357
:105F4C006F8F10BD38B5EFF31184202383F31288C3
:105F5C00BFF36F8F002390F86C50427B80F86C304D
:105F6C002DB121B184F31188BFF36F8F38BD12F0BE
:105F7C00280FF7D183680BB1FFF7A3FF437B23F006
:105F8C0004034373FDF7DCFAECE701211838FFF743
:105F9C00D9BF70B505460E46FDF7D2FCB6F1FF3FF2
:105FAC0008BFB5F1FF3F0446284612D04FF47A756E
:105FBC0047F61120002147F612220023C4FB0501ED
:105FCC00FAF756FAB0F1004F71F1000128BF6FF0EB
:105FDC00004070BD08B5C3171F3043F100034009E2
:105FEC0040EAC360C117FDF7ABFC400108BD2DE9C9
:105FFC00F04105460E461746EFF31188202383F334
:10600C001288BFF36F8F0468A0420FD1002088F371
:10601C001188BFF36F8FBDE8F08139462046B04739
:10602C000028F4D16B68A342F0D02468002CF4D182
:10603C00ECE708B50246FDF70BFE70B1D0E9043170
:10604C009B1A61EBE272B3F1004F72F1000104DABA
:10605C00002AACBF1846002008BD6FF00040FBE7DB
:10606C00024638B5EFF31185202383F31288BFF372
:10607C006F8F0368CBB1FDF7EBFD04461046FDF7BF
:10608C00F9FD00224FF000438442C0E9042306D1FD
:10609C00FDF7E6FDFFF7CDFF0021FCF7CFF8002060
:1060AC0085F31188BFF36F8F38BD6FF01500F7E7DC
:1060BC0008B5FDF7E9FE08BD704710B50446406A07
:1060CC0010B1A16A00F029F80020C4E9090010BD44
:1060DC0038B50546FFF7F1FF2B7F0446012B0ED098
:1060EC00023B012B0ED82B6A012B18BF6FF09604C4
:1060FC002C220021284600F057FA204638BD2B6A86
:10610C00002BF2E76FF09604F2E7FEF74FB87047FA
:10611C000020704700207047704710B5044608B146
:10612C00FDF7E2FF2046BDE81040FDF7D7BF0A2877
:10613C0040DCC31C22DA10F1400F47D010F13F0FA6
:10614C002BDA10F1410F44D010F1550F44D010F15F
:10615C00490F08BF6FF0840018BF6FF086007047BE
:10616C0009282AD8DFE800F005292908162938293A
:10617C00292F6FF09800704700207047C31C0D2B1F
:10618C001BD8DFE803F0072F1A1C1A1A1A1A1A1A4E
:10619C001D1A1A1D6FF08500704710F1210F1ED0CB
:1061AC000BDB10F1200F1DD010F1100F08BF6FF09A
:1061BC009400D1E764380928D2D96FF08600704773
:1061CC006FF0940070476FF08C0070476FF0840094
:1061DC0070476FF0890070476FF0930070476FF055
:1061EC00880070476FF09200704710B501380A4470
:1061FC00914200D110BD10F8013F11F8014B6340E2
:10620C000370F5E70144814200D1704711F8013D5C
:10621C001A440A70120AF6E710B58B4294BFC418E0
:10622C004418A04200D110BD00F8012BF9E700235F
:10623C001A4682B001908B4201D102B0704701988E
:10624C00C2540133F7E707B501A9FEF757F8003838
:10625C0018BF012003B05DF804FBF7B506460D46E8
:10626C00202D2F46A8BF202700216846FEF74EFBA5
:10627C00044670B93A4631466846FEF799FB10F170
:10628C00520F044608D0431CF4D0684600F0B5F811
:10629C0034B1204603B0F0BD684600F0AEF8E3E739
:1062AC00EC1B3E44F5D02546DAE7CA0448BF41F45E
:1062BC0080618B0448BF41F400618160704730B548
:1062CC0089B0054618220C4601A8002100F06CF993
:1062DC00012344EA052401A9BA2007940593FDF78C
:1062EC00C7FF002818BF6FF0920009B030BDF7B59A
:1062FC00BA2001A9FEF702F8044610B1002003B041
:10630C00F0BD019D2F0AEDB2AC4205D1BA20FDF7CC
:10631C00DBFF0028F2D008E0E6193046FDF7D4FF89
:10632C0030B13046FFF78FFF10B96FF09200E6E7FF
:10633C000134E9E708B5F820FFF785FF18B9F92013
:10634C00FFF781FF10B16FF0920008BDF820FDF748
:10635C00ADFF0028F7D1F920FDF7A8FF0028F4D0F5
:10636C00F1E738B5BFF35F8F4FF0A344E569BFF396
:10637C005F8FBFF35F8F10236363BFF35F8F0120C9
:10638C0000F092F8BFF35F8F00236363BFF35F8F5E
:10639C00BFF35F8FE36BBFF35F8F5B06F8D425B160
:1063AC00BFF35F8FE561BFF35F8F38BD08B5FEF7B4
:1063BC00F3FB30B9BFF35F8F4FF0A343986ABFF381
:1063CC005F8FBFF35F8F4FF0A342D36BBFF35F8F31
:1063DC0010F0240F03F0230304D0FFF7C2FF6FF07B
:1063EC001F0008BD4FF0FF30002BFAD1BFF35F8FB9
:1063FC001063BFF35F8F1846F3E710B503780446BC
:10640C001BB1FDF79DFE00232370002010BD02225E
:10641C0003689A607047C0F30B03482B4B6028BF8E
:10642C00482310F4003F8B6008BF0023CB6010F4AE
:10643C00803308BFC1E9013300F47003B3F5700F6A
:10644C0014BF00238B6800284FF0010C4FF008029A
:10645C008B60B8BF0023C1E905C2B8BFC1E90533E1
:10646C007047FCF75DBF4FF0FF324FF0FF33FCF786
:10647C00DFBE4FF0FF324FF0FF33FCF7D9BEFCF715
:10648C004FBF00F074B807B54FF0FF334FF0FF3239
:10649C00CDE90023002200F077F803B05DF804FB8F
:1064AC0000F06EB800F068B8FFF794BD2DE9F34723
:1064BC000446DDE90A9815460E4659B302F0010A66
:1064CC00FDF79EFA0746EFF31181202383F3128820
:1064DC00BFF36F8FA80744BF0023A360A36803EA30
:1064EC000600BAF1000F0CD086420CD16A0744BFEB
:1064FC008343A36081F31188BFF36F8F02B0BDE8B3
:10650C00F0870028F2D159EA080305D181F31188EC
:10651C00BFF36F8F0020F1E7C7E919652246CDE97B
:10652C00009804F10C00FDF7BDF80028F2D1786E4C
:10653C00E4E710B54B68D0E9194212F0010F03EAF9
:10654C00040301D09C4210D17BB14366520744BF77
:10655C008A681A430B6848BF8A6003660123086087
:10656C0080F86C301830FFF77BFD002010BD002345
:10657C00C0E90000836070474FF0FF32FEF756BB56
:10658C000A460021FEF752BB5200FFF78FBF0A44A8
:10659C00431E914200D1704710B511F8014B914246
:1065AC0003F8014FF9D110BD02440346934200D1C8
:1065BC00704703F8011BF9E70246014410B58A4203
:1065CC00134603D01C780132002CF8D1181A10BDD8
:1065DC00F0B5C3F13707044603F01F031046FFB2B2
:1065EC00082BE6B232D0102B3DD06508A40845EA42
:1065FC00C17544EA81748A082D1942EB51022909AC
:10660C0041EA02716D1842EB1212290A41EA026149
:10661C006D1842EB1222290C41EA02416D1842EB33
:10662C001242AD1842F10002EC0844EA4274D1085F
:10663C0004EB8402A6EB4205EDB2092D0CD9013412
:10664C00A5F10A0541F10001EDB212E0E40806F0F3
:10665C00070544EA4174C908303554EA010200F8D0
:10666C00015BBDD1F0BD240906F00F0544EA0174AD
:10667C000909092D84BFED19EDB2EDE70148006859
:08668C00704700000C0500201E
:086694001C9EFF7F01000000C5
:10669C00A917000000000000992100000000000074
:1066AC0000000000FC6600000000000034670000E1
:1066BC000000000018670000000000005067000098
:1066CC00000000006C670000911B0000000000003F
:1066DC00E3580000000000008517000000000000D7
:1066EC00EF58000000000000E90A00000000000064
:1066FC00A8760000E4700000247000004002002026
:10670C0048050020F918000000000000B5760000D4
:10671C000071000000700000420200209C05002067
:10672C00B51D000000000000C176000014710000CF
:10673C000070000044020020A8050020B51D0000D8
:10674C0000000000CC7600002871000000700000F2
:10675C0046020020B4050020B51D0000000000001A
:10676C00E0760000487100004070000048020020F4
:0C677C00C005002039580000000000009B
:10678800000000007B550000000000007B55000061
:10679800000000007B550000000000007B55000051
:1067A800000000007B550000000000007B55000041
:1067B800000000007B550000000000007B55000031
:1067C800000000007B550000000000007B55000021
:1067D800000000007B550000000000007B55000011
:1067E800000000007B550000000000007B55000001
:1067F800000000007B550000000000007B550000F1
:10680800000000007B550000000000007B550000E0
:10681800000000007B550000000000007B550000D0
:10682800000000007B550000000000007B550000C0
:10683800000000007B550000000000007B550000B0
:10684800000000007B550000000000007B550000A0
:10685800000000007B550000000000007B55000090
:10686800000000007B550000000000007B55000080
:10687800000000007B550000000000007B55000070
:10688800000000007B550000000000007B55000060
:10689800000000007B550000000000007B55000050
:1068A800000000007B550000000000007B55000040
:1068B800000000007B550000000000007B55000030
:1068C800000000007B550000000000007B55000020
:1068D800000000007B550000000000007B55000010
:1068E800000000007B550000000000007B55000000
:1068F800000000007B550000000000007B550000F0
:10690800000000007B550000000000007B550000DF
:10691800000000007B550000000000007B550000CF
:10692800000000007B550000000000007B550000BF
:10693800000000007B550000000000007B550000AF
:10694800000000007B550000000000007B5500009F
:10695800000000007B550000000000007B5500008F
:10696800000000007B550000000000007B5500007F
:10697800000000007B550000000000007B5500006F
:10698800000000007B550000000000007B5500005F
:10699800000000007B550000000000007B5500004F
:1069A800000000007B550000000000007B5500003F
:1069B800000000007B550000000000007B5500002F
:1069C80000000000154B0000000000007B5500008F
:1069D800000000007B550000000000007B5500000F
:1069E800000000007B550000000000007B550000FF
:1069F800000000007B550000000000007B550000EF
:106A0800000000007B550000000000007B550000DE
:106A1800000000007B550000000000007B550000CE
:106A2800000000007B550000000000007B550000BE
:106A3800000000007B550000000000007B550000AE
:106A4800000000007B550000000000007B5500009E
:106A5800000000007B550000000000007B5500008E
:106A6800000000007B550000000000007B5500007E
:106A7800000000007B550000000000007B5500006E
:106A8800000000007B550000000000007B5500005E
:106A9800000000007B550000000000007B5500004E
:106AA800000000007B550000000000007B5500003E
:106AB800000000007B550000000000007B5500002E
:106AC800000000007B550000000000007B5500001E
:106AD800000000007B550000000000007B5500000E
:106AE800000000007B550000000000007B550000FE
:106AF800000000007B550000000000007B550000EE
:106B0800000000007B550000000000007B550000DD
:106B1800000000007B550000000000007B550000CD
:106B2800000000007B550000000000007B550000BD
:106B3800000000007B550000000000007B550000AD
:106B4800000000007B550000000000007B5500009D
:106B5800000000007B550000000000007B5500008D
:106B6800000000007B550000000000007B5500007D
:106B7800000000007B550000000000007B5500006D
:106B8800000000007B550000000000007B5500005D
:106B9800000000007B550000000000007B5500004D
:106BA800000000007B550000000000007B5500003D
:106BB800000000007B550000000000007B5500002D
:106BC800000000007B550000000000007B5500001D
:106BD800000000007B550000000000007B5500000D
:106BE800000000007B550000000000007B550000FD
:106BF800000000007B550000000000007B550000ED
:106C0800000000007B550000000000007B550000DC
:106C1800000000007B550000000000007B550000CC
:106C2800000000007B550000000000007B550000BC
:106C3800000000007B550000000000007B550000AC
:106C4800000000007B550000000000007B5500009C
:106C5800000000007B550000000000007B5500008C
:106C6800000000007B550000000000007B5500007C
:106C7800000000007B550000000000007B5500006C
:106C8800000000007B550000000000007B5500005C
:106C9800000000007B550000000000007B5500004C
:106CA800000000007B550000000000007B5500003C
:106CB800000000007B550000000000007B5500002C
:106CC800000000007B550000000000007B5500001C
:106CD800000000007B550000000000007B5500000C
:106CE800000000007B550000000000007B550000FC
:106CF800000000007B550000000000007B550000EC
:106D0800000000007B550000000000007B550000DB
:106D1800000000007B550000000000007B550000CB
:106D2800000000007B550000000000007B550000BB
:106D3800000000007B550000000000007B550000AB
:106D4800000000007B550000000000007B5500009B
:106D5800000000007B550000000000007B5500008B
:106D6800000000007B550000000000007B5500007B
:106D7800000000007B550000000000007B5500006B
:106D8800000000007B550000000000007B5500005B
:106D9800000000007B550000000000007B5500004B
:106DA800000000007B550000000000007B5500003B
:106DB8006C670000DD570000000000007B550000F4
:106DC800000000007B550000000000007B5500001B
:106DD800000000007B550000000000007B5500000B
:106DE800000000007B550000000000007B550000FB
:106DF800000000007B550000000000007B550000EB
:106E0800000000007B550000000000007B550000DA
:106E1800000000007B550000000000007B550000CA
:106E2800000000007B550000000000007B550000BA
:106E3800000000007B550000000000007B550000AA
:106E4800000000007B550000000000007B5500009A
:106E5800000000007B5500007C010020B3570000B3
:106E6800000000007B550000000000007B5500007A
:106E7800000000007B550000000000007B5500006A
:106E8800000000007B550000000000007B5500005A
:106E9800000000007B550000000000007B5500004A
:106EA800212F00000D590000000000007B55000054
:106EB800000000007B550000000000007B5500002A
:106EC800000000007B550000000000007B5500001A
:106ED800000000007B550000000000007B5500000A
:106EE800000000007B550000000000007B550000FA
:106EF800000000007B550000000000007B550000EA
:106F0800000000007B550000000000007B550000D9
:106F1800000000007B550000000000007B550000C9
:106F2800000000007B550000000000007B550000B9
:106F3800000000007B550000000000007B550000A9
:106F4800000000007B550000000000007B55000099
:106F5800000000007B550000000000007B55000089
:106F6800000000007B550000000000007B55000079
:106F7800000000007B550000000000007B55000069
:106F8800000000007B550000000000007B55000059
:106F9800000000007B550000000000007B55000049
:106FA800000000007B550000A15900000D590000A9
:106FB800000000007B550000000000007B55000029
:106FC800000000007B550000000000007B55000019
:106FD800000000007B550000000000007B55000009
:106FE800000000007B55000004010020B35700009A
:086FF800000000007B550000C1
:10700000E11B000019570000255700003957000008
:10701000435700004D570000FD1D00006157000060
:04702000000000006C
:107024005119000089560000EB56000000000000D2
:0C703400255600000000000000000000D5
:0C704000F5570000A1200000E7570000F9
:1070500000A0105000820D500004055005000000F3
:10706000040000000100000000000000000000001B
:107070000338FDD870470000000000000000000049
:107080000338FDD8704700001867000001001100A8
:10709000346700000E000000506700000900000087
:1070A0006000002000000000060001000200000057
:1070B000B470000000000000997600000600000097
:1070C000E04F160000000020A17600002100000023
:1070D000E0EF0220F4000020B51800008518000041
:1070E00000000000051A0000851900001557000077
:1070F0001157000000A0105000820D5000040550F0
:107100007F00000000A010500401002000000000DB
:1071100000000000FFFF000000820D507C010020F5
:107120000000000001000000FF07000000040550FF
:1071300000000000000000000200000000A010504D
:1071400000820D500004055000600C50000000004B
:10715000000000007471000000C201000000D601B0
:107160000000000000000040000000004E0C002065
:107170004D0C002000600C508071000001000000E8
:1071800088710000040000002400000026000002B6
:10719000250600012706000300A0105000820D50B4
:1071A0000004055008000000020000000400000078
:1071B000010000009C660000AC660000DC66000078
:1071C000E4660000F4660000FC66000000010100B7
:1071D000000202000014000000280000004000002F
:1071E00001000000020000004F4E004F4646004CD8
:1071F00045442073746174653A2025730A002A2A75
:107200002A20426F6F74696E67206E524620436F6A
:107210006E6E6563742053444B2076332E332E30CC
:107220002D626131363764396633646234202A2A2C
:107230002A0A002A2A2A205573696E67205A657027
:10724000687972204F532076342E332E39392D66CB
:107250006439323034613032643532202A2A2A0AC5
:107260000072302F61313A20203078253038782074
:107270002072312F61323A20203078253038782042
:107280002072322F61333A20203078253038780A46
:107290000072332F61343A2020307825303878203E
:1072A0007231322F69703A202030782530387820BA
:1072B0007231342F6C723A20203078253038780AB9
:1072C0000020787073723A20203078253038780AA0
:1072D000004661756C74696E6720696E73747275AF
:1072E0006374696F6E2061646472657373202872C1
:1072F00031352F7063293A203078253038780A00EC
:10730000556E68616E646C6564204952516E3A2016
:1073100025640A002A2A2A2A2A2055534147452053
:107320004641554C54202A2A2A2A2A0A0020204461
:1073300069766973696F6E206279207A65726F0A67
:10734000002020556E616C69676E6564206D656D07
:107350006F7279206163636573730A002020537430
:1073600061636B206F766572666C6F772028636F40
:107370006E746578742061726561206E6F7420761A
:10738000616C6964290A0020204E6F20636F70725F
:107390006F636573736F7220696E73747275637453
:1073A000696F6E730A002020496C6C6567616C2000
:1073B0006C6F6164206F66204558435F5245545599
:1073C000524E20696E746F2050430A002020496C91
:1073D0006C6567616C20757365206F6620746865E5
:1073E00020455053520A002020417474656D70741A
:1073F00020746F206578656375746520756E6465AB
:1074000066696E656420696E737472756374696F02
:107410006E0A002A2A2A2A2A20425553204641551C
:107420004C54202A2A2A2A2A0A00202053746163F5
:107430006B696E67206572726F720A002020556E4C
:10744000737461636B696E67206572726F720A0094
:1074500020205072656369736520646174612062E5
:107460007573206572726F720A0020204246415285
:1074700020416464726573733A20307825780A007D
:107480002020496D70726563697365206461746161
:1074900020627573206572726F720A002020496E37
:1074A000737472756374696F6E2062757320657290
:1074B000726F720A002020466C6F6174696E672DCE
:1074C000706F696E74206C617A7920737461746571
:1074D00020707265736572766174696F6E20657273
:1074E000726F720A002A2A2A2A2A204D50552046F5
:1074F00041554C54202A2A2A2A2A0A002020537453
:1075000061636B696E67206572726F722028636FAA
:107510006E746578742061726561206D6967687446
:10752000206265206E6F742076616C6964290A00A0
:107530002020446174612041636365737320566940
:107540006F6C6174696F6E0A0020204D4D46415288
:1075500020416464726573733A20307825780A009C
:107560002020496E737472756374696F6E20416375
:10757000636573732056696F6C6174696F6E0A007E
:1075800052657365727665642045786365707469C9
:107590006F6E20280053707572696F757320696E65
:1075A00074657272757074202849525120005350CE
:1075B00053454C20696E20746872656164206D6F5C
:1075C000646520646F6573206E6F7420696E6469F2
:1075D00063617465205053500A002A2A2A2A2A20FF
:1075E00048415244204641554C54202A2A2A2A2AEE
:1075F0000A002020427573206661756C74206F6EDE
:1076000020766563746F72207461626C65207265A8
:1076100061640A0020204465627567206576656EA6
:10762000740A0020204661756C7420657363616C78
:107630006174696F6E20287365652062656C6F7771
:10764000290A00415243485F45584345505420772A
:1076500069746820726561736F6E2025780A0A006C
:107660002A2A2A2A2A204465627567206D6F6E696E
:10767000746F7220657863657074696F6E202A2A52
:107680002A2A2A0A002A2A2A2A2A2025732025643F
:1076900029202A2A2A2A2A0A00464C4153485F30C8
:1076A000005352414D5F3000636C6F636B4031306B
:1076B00065303030006770696F4031306130303094
:1076C000006770696F406438323030006770696FEE
:1076D0004035303430300000010405020608090F3F
:1076E0007561727440633630303000000718232310
:1076F00023232323232323232323230001026D6138
:10770000696E00286E756C6C29002A666C6F617456
:047710002A0000004B
:1077140000000000670000000000000000000000FE
:107724000000000000000000000000000000000055
:107734000000000000000000000000000000000045
:107744000000000000000000000000000000000035
:107754000000000000000000000000000000000025
:107764000000000000000000000000000000000015
:107774000000000000000000000000000000000005
:1077840000000000000000000000000000000000F5
:1077940000000000000000000000000000000000E5
:1077A4008F530000000000001B5600000000000082
:1077B4000000000000C010500000000000000000A5
:1077C40000000000000000000000000000000000B5
:1077D40000000000000000000000000000000000A5
:1077E4000000000000000000000000000000000095
:1077F4000000000000000000000000000000000085
:107804000000000000000000000000000000000074
:107814000000000000000000000000000000000064
:1078240000000000000000000001000000A00D5056
:107834000000000000000000000000000000000044
:107844000000000000000000000000000000000034
:107854000000000000000000000000000000000024
:107864000000000000000000000000000000000014
:107874000000000000000000000000000000000004
:1078840000000000000000000000000000000000F4
:1078940000000000000000000000000000000000E4
:1078A400000000005521000000000000FF0000005F
:1078B4000090D003FF0000000F00000071020000E0
:1078C400100200201002002025610000B5650000B0
:1078D400677420004C020020740200206002002023
:1078E400BC020020B00200206F640000736400003A
:0C78F40000000000000000000000000088
:107900004C0200204C02002000000000000000009B
:107910000E00000060020020600200200000000055
:10792000000000000E00000074020020740200201D
:1079300000000000000000000E000000880200208F
:107940008802002000000000000000000E0000007F
:107950009C0200209C0200200000000000000000AB
:047960000E00000015
:10796400B0020020B002002000000000BC02002091
:08797400BC020020000000002D
:04797C0015E015E01D
:040000030000100DDC
:00000001FF
